:100000000C94D1030C9418040C9418040C94B71B92
:100010000C9418040C9418040C9418040C941804F0
:100020000C9418040C9418040C949A2A0C945029DB
:100030000C9485210C9418040C9418040C94180446
:100040000C9418040C94C0110C9418040C9418040B
:100050000C9418040C9429210C9418040C94180482
:100060000C9418040C9418040C9418040C941804A0
:100070000C9418040C9418040C9418040C94180490
:100080000C9418040C9418040C9418040C94180480
:100090000C94081C0C9418040C9418040C94180468
:1000A0000C9418040C9418040C9418043F0841088C
:1000B00043084508470849084B084D0856085808A2
:1000C0005A085C085E0860086208640866087108DF
:1000D000DB08DB08160916095609110B110B110B69
:1000E0007609110B730A730A800A800A800A800A53
:1000F000800A800A800A800A800A800A800A800AB0
:10010000800A800A800A800A8F0AB80ABD0AC40AD7
:10011000DC0A61278827282988272829D027F32760
:100120002829F1280429E82BE82BFB2BFB2BF12BAA
:10013000FB2BFB2BFB2BE82BE82BF62BFB2BFB2BBA
:10014000F62B07634236B79BD8A71A39685618AE04
:10015000BAAB558C1D3CB7CC5763BD6DEDFD753EFC
:10016000F6177231BF000000803F05A84CCDB2D415
:100170004EB93836A9020C50B9918688083CA6AA17
:10018000AA2ABE000000803F08000000BE92244959
:10019000123EABAAAA2ABECDCCCC4C3E00000080B9
:1001A000BEABAAAAAA3E00000000BF000000803F2C
:1001B0000000000000084178D3BB4387D1133D19EC
:1001C0000E3CC3BD4282AD2B3E68EC8276BED98F19
:1001D000E1A93E4C80EFFFBE01C4FF7F3F0000005D
:1001E00000002B0014001A00080015001700000082
:1001F000E00004001600070009000A000000E1000A
:100200001D001B000600190005000000EA5C290023
:10021000E200E300EC5CE85C2C002A001300120012
:100220000C0018001C000000340033000F000E000A
:100230000D000B00000028003800370036001000C9
:10024000110000004F00520051005000ED5CE95CCD
:100250002C002B0014001A00090013000A000000F3
:10026000E000040015001600170007000000E10080
:100270001D001B000600190005000000EA5C2900B3
:10028000E200E300EC5CE85C2C002A0033001C0078
:1002900018000F000D000000340012000C000800D0
:1002A00011000B0000002800380037003600100055
:1002B0000E0000004F00520051005000ED5CE95C60
:1002C0002C002B0034003600370013001C00000007
:1002D000E00004001200080018000C000000E1001B
:1002E000330014000D000E001B000000EA5C290022
:1002F000E200E300EC5CE85C2C002A000F00150033
:1003000006000A000900000038001600110017005E
:100310000B000700000028001D0019001A00100043
:10032000050000004F00520051005000ED5CE95CF8
:100330002C0035021E021F022002210222020000B0
:1003400001003A003B003C003D003E00000001007F
:100350004000410042004300440000000100010051
:10036000010001000100010001004C0027022602EB
:100370002502240223020000310230022F022E0245
:100380002D023F00000001004D004A004600010020
:1003900045000000AE00A900AA00AB00010001006A
:1003A000010035001E001F00200021002200000077
:1003B00001003A003B003C003D003E00000001000F
:1003C00040004100420043004400000001000100E1
:1003D000010001000100010001004C00270026007F
:1003E0002500240023000000310030002F002E00E3
:1003F0002D003F00000001004B004E0046000100B0
:1004000045000000AE00A900AA00AB0001000100F9
:1004100001000100005C010001000100010000007A
:1004200001001D5C1E5C285C295C135C000001005F
:10043000205C255C235C245C0100000001000100BD
:1004400001000100010001000100010001000100A4
:10045000010001000100000001000100E75CE65C12
:10046000E55C0A5C0000C95CC75CC55CC25C01005D
:1004700001000000CA5CC85CC65CC35C01000100EE
:10048000010002E26003E20002E26003E200000019
:10049000000000000000000000000000000000005C
:1004A000000000000000000000000000000000014B
:1004B0000101010101000101010100000000000033
:1004C0000000000000000000010001000101010126
:1004D000010101010101010101010101010101010C
:1004E0000101010101010101010000000101000001
:1004F00000000000000000000000000000000000FC
:1005000000000000000000000001010101000000E7
:100510000000000000002A2B28000000000000005E
:1005200000000000000000000029000000002C1E58
:100530003420212224342627252E362D3738271E15
:100540001F202122232425263333362E37381F043B
:1005500005060708090A0B0C0D0E0F1011121314D3
:1005600015161718191A1B1C1D2F3130232D350491
:1005700005060708090A0B0C0D0E0F1011121314B3
:1005800015161718191A1B1C1D2F3130354C000079
:10059000000000010101010101010101020202024A
:1005A000020202020203030303030303030404041D
:1005B00004040405050505050606060606070707E3
:1005C00007080808080909090A0A0A0A0B0B0B0C94
:1005D0000C0C0D0D0D0E0E0F0F0F1010111111122E
:1005E0001213131414151516161717181819191AAB
:1005F0001A1B1C1C1D1D1E1F1F202021222223240C
:10060000252526272728292A2B2B2C2D2E2F2F3046
:10061000313233343536363738393A3B3C3D3E3F5C
:100620004041424344464748494A4B4C4D4F505144
:100630005253555657585A5B5C5E5F6062636466FE
:1006400067696A6C6D6E707173747678797B7C7E85
:100650008081838486888A8B8D8F91929496989AD4
:100660009B9D9FA1A3A5A7A9ABADAFB1B3B5B7B9EA
:10067000BBBDBFC1C4C6C8CACCCFD1D3D6D8DADCC3
:10068000DFE1E4E6E8EBEDF0F2F5F7FAFCFF6801F4
:10069000F000B40078005A001E140A05783C1E646D
:1006A00032146432147F3F1F05010980A1018503C4
:1006B0001601002603001A81002A83007510950197
:1006C0008100C0050C0901A1018504160100269CCA
:1006D000021A01002A9C02751095018100C00501D3
:1006E0000906A101050719E029E71500250195086C
:1006F0007501810295017508810105081901290517
:100700009505750191029501750391010507190081
:1007100029FF150026FF00950675088100C0090213
:100720003B00020100A0C809040000010301010010
:100730000921110100012240000705810308000A78
:100740000904010001030000000921110100012238
:1007500036000705820320000A1201100100000084
:1007600008EDFE60300200010203010403300000C6
:10077000001403480065006C0069007800500069AF
:100780000063006F000000140359007500730068D7
:100790000061006B006F0062006F0000000403093D
:1007A000040011241FBECFEFDAE0DEBFCDBF04B6D8
:1007B00003FE27C08091010690910206A0910306D6
:1007C000B09104068730904BA740B04BD1F4109203
:1007D000010610920206109203061092040614BE3F
:1007E00084B7877F84BF0FB6F894A8958091600086
:1007F000886180936000109260000FBEE0E0F8E333
:10080000099514E0A0E0B1E0ECE0F5E602C0059047
:100810000D92A438B107D9F726E0A4E8B4E001C0EE
:100820001D92A130B207E1F70E94171D0C9484328B
:100830000C9400004F925F926F927F92AF92BF92A2
:10084000CF92DF92EF92FF920F931F93CF93DF939C
:10085000CDB7DEB7A4970FB6F894DEBF0FBECDBFFD
:10086000FC01B080118183819481892B11F40C9457
:10087000250E1F3F29F40FEFB01611F40C94250E2E
:100880007F01C080D1808281882349F0C6010E9407
:100890004722082F682FC6010E94BF2204C0C6014C
:1008A0000E949322082F27E0129FF001112438E3C1
:1008B000039FE00DF11D1124EB0DF11DEE0FFF1F45
:1008C000EE51FE4F0591149100328CE5180781F42A
:1008D000D70112968C91882309F46AC06091FE05B5
:1008E00061FB992790F981E0892780FB61F90CC0B1
:1008F0000132BCE51B0779F4F7018281882309F4F2
:1009000057C06091FE0562606093FE0587E090E04D
:100910000E949B2D4DC00232FCE51F0781F4D701D8
:1009200012968C91882309F46BC06091FE056D7F4F
:100930006093FE0587E090E00E949B2D61C0053228
:10094000BCE51B0791F4F7018281882309F458C0A4
:1009500080E090E0ACEDB3E4809314019093150136
:10096000A0931601B09317014BC00332FCE51F079B
:10097000F9F4D70112968C91882309F441C029E03B
:1009800038E348E95FE360911401709115018091AB
:100990001601909117010E94D3302B013C0120E0F9
:1009A00030E84BEB54E40E949F2E87FF29C020C003
:1009B0000432BCE51B0721F5F7018281882301F190
:1009C00029E038E348E95FE3609114017091150173
:1009D00080911601909117010E94A42E2B013C01D9
:1009E00020E030E042E852E40E945830181644F407
:1009F00040921401509215016092160170921701F5
:100A00008091FE0581FF7AC0D70112968C918823D0
:100A100009F489C080919E048111BBC080919D041E
:100A20008111B7C060911401709115018091160178
:100A3000909117019B01AC010E94332E2B013C01C8
:100A40000E94772DBC01990F880B990B0E94812F72
:100A500020E03EEF4FEF56E40E94A42E2DEC3CEC3C
:100A60004CE45DE30E94D33020E030E040E85FE3F7
:100A70000E94332E9B01AC01C301B2010E94D3300E
:100A80006093040170930501809306019093070120
:100A9000409014015090150160901601709017015C
:100AA0000E94772DBC01990F880B990B0E94812F12
:100AB00020E03EEF4FEF56E40E94A42E2DEC3CECDC
:100AC0004CE45DE30E94D33020E030E040E85FE397
:100AD0000E94332E9B01AC01C301B2010E94D330AE
:100AE00060930C0170930D0180930E0190930F01A0
:100AF00062E070E084E091E00E94AC25083EBCE535
:100B00001B0709F44BC010F00C94B60D053EFCE534
:100B10001F0799F010F00C94060E033C3CE51307F8
:100B200009F475C092C0083E2CE51207B9F108F02F
:100B300048C0053E8CE5180781F4D70112968C91C8
:100B4000882311F40C94250E64E070E088E891E0AD
:100B50000E94AC2581E090E018C0063E9CE5190794
:100B600008F46DC0063EBCE51B0709F0E6C7F701B7
:100B70008281882311F40C94250E66E070E088E5EC
:100B800091E00E94AC2582E090E00E94111A0C9442
:100B9000250E083EBCE51B0709F0E3C7F70182817B
:100BA000882349F080918404811103C081E08093FF
:100BB000840483E020C01092840483E00E94F82221
:100BC00022C00C3EFCE51F0709F4D4C708F09EC004
:100BD000093E3CE5130711F00C94E50DD701129680
:100BE0008C91882359F080918404811103C081E0A5
:100BF0008093840484E00E94342305C084E00E9432
:100C0000F822109284040E940E260C94250ED7011F
:100C100012968C91882311F40C94250E8091130563
:100C20000E9457110E94641180914A0586958F7326
:100C300090E090931405809313050C94250E033CCB
:100C4000ACE51A0711F40C94250E0D31BCE51B0719
:100C500051F4D70112968C91882309F479C00E942F
:100C6000B1110C94250E0E31BCE51B0741F4F701C0
:100C70008281882309F46CC00E94AA15E6C70F314F
:100C8000FCE51F0759F4D70112968C91882309F4CB
:100C90005FC08091FE0580FDEFCFE1CFC8018A5291
:100CA0009C45029760F4F7018281882309F450C0C3
:100CB0001092850464E070E088EA91E024C0063276
:100CC000ECE51E0709F40EC10732BCE51B0709F469
:100CD00012C10832FCE51F0709F415C10C32BCE54E
:100CE0001B0709F41BC10D32FCE51F0709F01EC1EB
:100CF000D70112968C91882359F110929D0468E0D7
:100D000070E088EC91E00E94AC259FC70D3E9CE509
:100D1000190709F448C70E3EACE51A0709F095CF4C
:100D2000F70182818823A1F00E94C60F80914A05B5
:100D3000816080934A0586958F730E945711809138
:100D40004A0586958F7390E0909314058093130560
:100D500090919E04911105C080919D04882309F40F
:100D600014C1F7016281662309F44BC0003E1105EE
:100D700061F40E949A1581E080939C0410929B0478
:100D800010929A041092990460C7023E110571F402
:100D90000E949A1580919C04882319F081E0809329
:100DA0009B0410929C0410929A044FC7033E1105B5
:100DB00091F480919B04882321F10E949A1510924E
:100DC0009C0481E080939A041092980410929704F6
:100DD000109296043AC70235110531F48091A902A8
:100DE0009091AA020A9708C00135110551F480912B
:100DF000A9029091AA020A969093AA028093A9024E
:100E000024C78091A80281110BC0D7012C91205FCB
:100E100011968C9148E050E0481B5109BCE01DC080
:100E2000813079F4F701208183E3820F418128E04A
:100E300030E0241B3109322F330F330F230F280FDB
:100E40002FC0823071F4D7012C912D5C11968C91BA
:100E500048E050E0481B5109B7E04B9F200D11249A
:100E60001FC08330E1F483E2E2E5F4E0DE01119695
:100E700001900D928A95E1F7F7018081FE01E80F5C
:100E8000F11DD70111968C9148E050E0481B5109A3
:100E90002085BCE04B9F200D1124275F01C02CE072
:100EA0006623B1F0992329F0822F2CA30E949F166C
:100EB0002CA180919C04882381F080919904E82FD3
:100EC000F0E0EA57FB4F20838F5F8093990405C0C1
:100ED000992319F0822F0E94C4150F3F110508F0C5
:100EE00054C0B3C6D70112968C91882309F430CF31
:100EF0000E94A211AAC6F7018281882309F428CF93
:100F00000E94A015A2C6D70112968C91882309F4DD
:100F10001FCF80919E048111F3CFEACFF701828128
:100F2000882309F415CF0E9499118FC60E32BCE5B3
:100F30001B0751F4F7018281882309F409CF8091BE
:100F40009D048111DACEEFCF0932FCE51F0709F0CD
:100F5000FFCED70112968C91882309F4F9CE0E9416
:100F60009A152091A80230E02F5F3F4F237033275E
:100F70002093A80248E2429FC001439F900D112494
:100F800065E070E0885F9D4FBECE0C3CFCE51F071E
:100F9000F9F4F7018281882309F457C680914E0540
:100FA00090E0019797FF02C080E090E084309105C7
:100FB00014F083E090E080934E0560914A057091B3
:100FC0004B0580914C0590914D050E94A80F3DC6A0
:100FD0000D3C2CE5120708F0CDC3D70112968C9179
:100FE000043CBCE51B0751F4882309F42EC680910C
:100FF000BB058272D1F40E945A1127C6053CECE56C
:101000001E0708F003C40531FCE51F0788F0023C09
:10101000ACE51A0709F486C308F4CBC3882309F4A6
:1010200014C68091BB05827231F70E9464110DC60F
:1010300002302CE5120708F468C0882309F473C055
:101040000E94C821811102C00E94D32184E090E057
:101050000E94872D90E090931F0580931E05F80154
:10106000E350FC45E231F10530F4EA5AFF4F80913C
:101070001E050C94713280911E05816039C082601A
:1010800037C0846035C0886033C0806131C0806201
:101090002FC080642DC080682BC0846088608093DE
:1010A0001E0564E070E083ED92E018C08E7F20C0E2
:1010B0008D7F1EC08B7F1CC0877F1AC08F7E18C09B
:1010C0008F7D16C08F7B14C08F7712C08B7F877F78
:1010D00080931E0562E070E083EC92E00E94AC25F4
:1010E00009C087FB222720F991E0922790FB87F91E
:1010F00080931E0560911E0584E090E00E949B2D68
:101100001092BB050E940D2CA0C501153CE51307EC
:1011100009F4C2C201301C4509F4FBC281E080938E
:10112000A4048093A504D70112968C9112970D9177
:101130001C91882349F0C8010E944722D82E682FAD
:10114000C8010E94BF2204C0C8010E949322D82E69
:10115000B8018D2D0E948117182F782EF701058177
:1011600002950F70B280B1101092B6058091B30550
:10117000877089F0BB2079F080E2810F883058F0C9
:1011800082E09CA30E941D238091B3058770AA244E
:10119000A3949CA18111A12CC92EC2948FE0C822D6
:1011A000D12CFCE0CF16D10408F03BC2F601E8597F
:1011B000FF4F0C947132892F807F9F70092F8823F5
:1011C00011F00295007FBB20B9F0002309F414C28E
:1011D00080E2810F883010F0711006C09091BB053D
:1011E000092B0093BB0505C09091B605092B009310
:1011F000B6050E94192200C2812F0E942B2C0023C9
:1012000009F40FC2105E0095183010F0711006C07E
:101210009091BB0509230093BB0505C09091B605CD
:1012200009230093B6050E941922FBC1292F207FB4
:10123000892F8F70203211F08295807F772021F0E6
:1012400021E07216A9F01EC0BB2051F09091B405A8
:10125000892B002321F1013011F58093B405E1C100
:10126000002319F0013009F4DCC11092B40554C117
:10127000BB2021F0063008F0D4C111C0053008F0C1
:10128000D0C14AC1BB2071F0002349F0D7011596A7
:101290009C91159790FFB0C19F7015969C930E94EA
:1012A000212CBFC1002309F437C1B8C1292F2695CD
:1012B0002695237030E02115310521F021303105CC
:1012C00059F0AFC1BB2019F0812F937002C080E0AC
:1012D00090E00E94610FB3C1BB2019F0812F937081
:1012E00002C080E090E00E944B0FA9C1892F83705B
:1012F00009F079C0B110A1C1812F829586958770C0
:10130000880F880F412F4F7050E060E070E02A0195
:101310003B01082E04C0440C551C661C771C0A9423
:10132000D2F714FF14C04FE050E060E070E08A0193
:101330009B0104C0000F111F221F331F8A95D2F793
:10134000B901A801409550956095709503C040E0A3
:1013500050E0BA01969596959370892F90E0009190
:10136000B7051091B8052091B9053091BA058230C2
:101370009105A9F083309105E9F0019759F04429CE
:10138000552966297729CB01BA016023712382236D
:10139000932326C0402A512A622A732A1BC044295B
:1013A000552966297729CB01BA0160277127822741
:1013B000932716C0CB01BA016023712382239323A4
:1013C0000E9455234091B7055091B8056091B90529
:1013D0007091BA05CB01BA0164297529862997292C
:1013E0000E9455232AC1BB2019F0892F817001C0AA
:1013F0008695882309F421C1812F8295869587706F
:10140000880F880F412F4F7050E060E070E02A0194
:101410003B01082E04C0440C551C661C771C0A9422
:10142000D2F714FF14C04FE050E060E070E08A0192
:101430009B0104C0000F111F221F331F8A95D2F792
:10144000B901A801409550956095709503C040E0A2
:1014500050E0BA01969596959370892F90E000918F
:10146000E4051091E5052091E6053091E70582300D
:101470009105A9F083309105E9F0019759F04429CD
:10148000552966297729CB01BA016023712382236C
:10149000932326C0402A512A622A732A1BC044295A
:1014A000552966297729CB01BA0160277127822740
:1014B000932716C0CB01BA016023712382239323A3
:1014C0000E94EE224091E4055091E5056091E60509
:1014D0007091E705CB01BA016429752986299729FE
:1014E0000E94EE22AAC0412F50E0FA01E05EF1090D
:1014F000E531F10508F07BC0EC58FF4F0C947132D8
:101500001F70892F8F71BB2021F00E943423812FFF
:10151000C6CE0E94F822812F0E94162C82C0BB20CA
:1015200019F1053008F07DC0292F2F7181E090E07E
:10153000A0E0B0E0AC01BD0104C0440F551F661F20
:10154000771F2A95D2F78091E4059091E505A09147
:10155000E605B091E7058A019B01082719272A278C
:101560003B27C901B80125C0063008F05AC0DCCFBE
:10157000BB2029F0892F8F712EC0BB20D9F3892F72
:101580008F710E94F8224DC0BB2081F0292F2F714E
:1015900081E090E0A0E0B0E0BC01CD0104C0660FA6
:1015A000771F881F991F2A95D2F703C060E070E06B
:1015B000CB010E94EE2235C0BB2081F0192F1F7194
:1015C000812F0E94342328E0129FC00111248360E0
:1015D0008093B305812F0E94342323C081E00E94B1
:1015E0001D230230F0F082E00E941D231AC0BB20B0
:1015F00039F0002309F4BECF812F0E94632C11C063
:10160000002309F4BCCF193349F43FEF87EE93E090
:10161000315080409040E1F700C00000812F0E94CF
:101620002B2CA8E0CA16D10441F04CF0EAE0CE1A07
:10163000D108F2E0CF16D10410F40E94770FAA204F
:1016400009F403C38091B30580FDFFC2D701129650
:101650001C928595859585950E943423C7010E942B
:101660001A048091B305859585958595A4960FB646
:10167000F894DEBF0FBECDBFDF91CF911F910F91C8
:10168000FF90EF90DF90CF90BF90AF907F906F90E2
:101690005F904F900C94F822882309F4D6C21092E0
:1016A000BB050E940D2C0E949A150E9479218C0185
:1016B00063E070E08BEA92E00E94AC25EFEFF2E588
:1016C00027E0E150F0402040E1F700C000000E9418
:1016D0005F15C8010E944F218A3F910538F48FE9B8
:1016E0009FE00197F1F700C00000F3CF0E945F1563
:1016F00087E797E790930108809300089AE088E1D4
:101700000FB6F894A895809360000FBE9093600088
:10171000FFCF882309F499C280912C0581608093C2
:101720002C0593C2882309F490C280914A0580FF5A
:101730001BC08E7F80934A0560914A0570914B05CE
:1017400080914C0590914D050E94A80F10924F0575
:101750009FEFA0E7B2E09150A040B040E1F700C099
:1017600000000E94830F71C2816080934A058695B4
:101770008F731CC0043DECE51E0709F4F2C008F0AD
:1017800041C1D70112968C91003DBCE51B0709F4BD
:10179000F6C008F015C10E3CFCE51F0709F4FAC0BD
:1017A00008F003C1882309F450C281E00E94571158
:1017B0004CC206311C4509F0B1CC9091BB05882381
:1017C00081F09A7A81E009F480E080939F0481118E
:1017D00002C069E201C065E380E595E00E94AE21A8
:1017E00012C080919F04811102C089E201C085E38B
:1017F000E2E5F5E096E09E0F2081281301C01082FB
:1018000031969E13F9CF0E9419221FC2083CFCE5B5
:101810001F07F9F4882309F418C260914C05862F3C
:1018200090E04197A4F0615180914A05881F882774
:10183000881F90914B05392F330F97FB992790F90B
:1018400021E040914D05832B0E944A10FEC160E0CB
:10185000EBCF093C2CE5120708F04AC0063C3CE5FA
:10186000130711F5882309F4F0C120914A05221FBE
:101870002227221F30914B05432F440F842F822BA8
:1018800037FB992790F98A3091051CF4825A9E4FB4
:1018900001C00A9768E671E00E945D3221E0409144
:1018A0004D0560914C05D0CF073C1C4598F488232A
:1018B00009F4CBC120914A05221F2227221F309113
:1018C0004B05432F440F842F822B37FB992790F928
:1018D0000A96E0CF882309F4B8C160914C05862FA1
:1018E00090E08F3E910514F46F5E9ECF6FEF9CCF1A
:1018F0000A3CACE51A07E1F4882309F4A6C140913B
:101900004D05842F90E0419714F0415101C040E013
:1019100080914A05881F8827881F90914B05392F91
:10192000330F97FB992790F921E060914C058BCFFD
:101930000B3C1C4570F4882309F487C140914D0588
:10194000842F90E08F3E910514F44F5EE1CF4FEF6E
:10195000DFCF882309F479C180914E0590E001968C
:1019600025CBD70112968C91882309F46EC10E9471
:101970009F0F8951893008F458CB89E117CF88230C
:1019800009F463C10E949F0F8950853008F44DCB44
:1019900089E00CCF882309F458C10E949F0F825020
:1019A000833008F442CB82E001CF882309F44DC193
:1019B0000E949F0F8650823008F437CB86E0F6CE27
:1019C000023D3CE5130759F4882309F43EC10E9407
:1019D0009F0F8551823008F428CB85E1E7CE033D87
:1019E0001C4558F4882309F430C10E949F0F8F5082
:1019F000853008F41ACB8FE0D9CE882309F425C1AD
:101A000088E1D4CE083DACE51A0759F5F70182818B
:101A1000882361F01092A5040E9479219093A30479
:101A20008093A20480E20E94212C0FC18091A50422
:101A3000882321F080E20E94162C07C18091A20425
:101A40009091A3040E944F218436910598F780E27B
:101A50000E94162C88E20E94632C88E20E942B2CA4
:101A6000F4C0093DBCE51B0708F045C0063DECE5A8
:101A70001E0719F5F7018281882351F01092A40402
:101A80000E9479219093A1048093A00482E0CBCF9F
:101A90008091A40481110FC08091A0049091A104B1
:101AA0000E944F218436910530F486E20E94632C17
:101AB00086E20E942B2C82E0BECF073D1C4508F435
:101AC000C4C0D70112968C918111A4CF8091A50436
:101AD0008111B0CF8091A2049091A3040E944F2164
:101AE0008436910508F0A6CF87E20E94632C87E236
:101AF0000E942B2C9FCFD70112968C910C3DBCE5F8
:101B00001B0739F4882309F4A0C082E080930F05F5
:101B10009CC00D3DECE51E0731F4882309F495C007
:101B20000E94D32192C00B3D1C4509F0F7CA8823BF
:101B300009F48BC010920F0588C0073EECE51E0724
:101B400009F083C8D70112968C91882309F47DC0CF
:101B500068E070E088E191E00E94AC2584E090E0CC
:101B600014C8093EECE51E0708F442C00C3EACE583
:101B70001A0779F4F7018281882349F080911E05C4
:101B800082FD02C081E919C088E894E01BC081E9A8
:101B900065CF0D3EBCE51B0708F444C00D3E2CE5A7
:101BA000120709F04BC0D70112968C918823F1F0EF
:101BB00080911E0582FD04C080E90E94632C45C00F
:101BC00082E894E00E94D01940C00A3E8CE51807D4
:101BD00009F03BC8F7018281882321F085E00E944B
:101BE000342333C085E00E94F8222FC080E936CF2D
:101BF000053EFCE51F0711F40C94A40538F4033CE2
:101C00003CE5130711F40C940E061FC8063E8CE544
:101C1000180711F40C94B705073E9CE5190709F461
:101C200091CF13C8093EECE51E0711F40C94EE05A4
:101C30000A3EFCE51F0771F20C9425060E3E3CE5BA
:101C4000130709F46DC80C942506A4960FB6F894F2
:101C5000DEBF0FBECDBFDF91CF911F910F91FF90DF
:101C6000EF90DF90CF90BF90AF907F906F905F909C
:101C70004F90089590911E0592FF0DC0282F287156
:101C8000283019F4877F846006C0282F24712430FF
:101C900011F48B7F886093FF0DC0282F28712831A5
:101CA00019F4877E846106C0282F2471243111F431
:101CB0008B7E886194FD877E08958EE14A9B02C0E9
:101CC0008150E1F74A9BFECF08955A9880E28A95A9
:101CD000F1F75A9A0895FF920F931F93CF93DF93D2
:101CE00000D0CDB7DEB71982F82E8C01802F8F1966
:101CF000861760F46A830E945D0ECE0101960E94F1
:101D00006725F80181938F016A81F0CF81E0998185
:101D1000911180E00F900F90DF91CF911F910F9163
:101D2000FF900895EF92FF921F93CF93DF9300D01F
:101D3000CDB7DEB7182F7C018E2D811B861760F47E
:101D4000F70181917F016A8389830E94650E8981F1
:101D50000E948F256A81F0CF0F900F90DF91CF9175
:101D60001F91FF90EF9008951F93CF93DF93CDB70E
:101D7000DEB767970FB6F894DEBF0FBECDBF4B8BB3
:101D80005C8B6D8B7E8B8F8B86E09E01235F3F4F3C
:101D9000D901E82F1D92EA95E9F795E0FE017396C7
:101DA000D90101900D929A95E1F7F901DE0117969C
:101DB00001900D928A95E1F7CE0107960E94C42307
:101DC000811136C086E0FE013796DE011196019042
:101DD0000D928A95E1F77F816885EA85FB853097CA
:101DE00039F16F3F11F47F3F19F120915E0530E02A
:101DF000C90101968770992740918F0550E084179B
:101E0000950779F179836A83FD83EC8396E0929F4D
:101E1000D001939FB00D1124A15ABA4FFE01319603
:101E200001900D929A95E1F780935E050E945F23E1
:101E300016E080918F0590915E05891711F1189F2A
:101E4000C0011124815A9A4F0E94C4238823C9F0EB
:101E500080918F0590E001968770992780938F0578
:101E6000E8CF1092BB050E940D2C10925E051092D7
:101E70008F05E8E5F5E086E0DF011D928A95E9F738
:101E8000D7CF67960FB6F894DEBF0FBECDBFDF91F8
:101E9000CF911F910895209100053091010582177F
:101EA000930771F09093010580930005E091200560
:101EB000F0912105309721F00084F185E02D0994FF
:101EC00008952091FE043091FF048217930771F06A
:101ED0009093FF048093FE04E0912005F09121058A
:101EE000309721F00680F781E02D09940895E09164
:101EF0002005F0912105309721F00190F081E02D2F
:101F0000099480E0089580914A0580FD0CC080E02E
:101F100090E0FC01EE52FA4F118210821282039679
:101F200082319105B1F7539A82E190E00E94242614
:101F300087EC90E00197F1F700C0000008958091D0
:101F40004A0580FF03C086958F73089580E0089549
:101F5000CF92DF92EF92FF926B017C0188E090E0DC
:101F60000E948F2D6C157D058E059F0551F0B701E0
:101F7000A60188E090E0FF90EF90DF90CF900C9466
:101F8000AD2DFF90EF90DF90CF900895EAE4F5E05B
:101F900083E0808310924B058FEF828383831482CA
:101FA00060817181828193810C94A80FEF92FF92DE
:101FB0000F931F93CF93DF93E901662309F44BC07E
:101FC000242F30E0EFEFF0E0E61BF109B901E69FC6
:101FD0009001E79F300DF69F300D1124232F8B01C8
:101FE000031B11095CE3E52EF12CB7010E94493275
:101FF000FB01BC01069FC001079F900D169F900D2D
:102000001124B7010E944932E230F105B1F040F4E9
:10201000309779F0319711F5832F242F461B21C07B
:10202000E430F105A1F068F03597C1F4842F861BE8
:1020300018C0832F262F230F14C0862F830FE42F61
:1020400003C0E42FE61B842F432F2E2F0AC0842FBA
:10205000462F430F06C0842F242F03C080E020E0CA
:1020600040E0E42FF0E0E257FA4F4491E22FF0E035
:10207000E257FA4F9491E82FF0E0E257FA4FE491DB
:1020800049839883EA83DF91CF911F910F91FF904D
:10209000EF9008955F926F927F928F929F92AF928E
:1020A000BF92CF92DF92EF92FF920F931F93CF9345
:1020B000DF9300D01F92CDB7DEB78C01E62EF42E51
:1020C000522E80914A0580FF97C0982F9E779230BC
:1020D000D1F49E012F5F3F4FC8010E94D60F2B8184
:1020E00039814A8180914A0580FF66C080E090E096
:1020F000FC01EE52FA4F41833083228303968231F2
:102100009105B1F757C0E82FE695EF739EE39E0F58
:102110009F73943018F4F0904D054EC09AE39E0FD3
:102120009F73993068F4881F8827881F90914B050A
:10213000292F220F022F082B97FB112710F93CC0E3
:1021400087E28E0F8F738A30B8F5F0E07997E0FD63
:1021500002C021E001C02FEFEE7FE257F94F8591D9
:10216000949166E070E00E94493226034001279F67
:10217000900C1124580188E9A81A8EEFB80A82ED54
:10218000C82E85E0D82E98E6692E77247394C50171
:10219000B3010E94493296014F2D6E2D0E94D60F39
:1021A000A80CB91C83E0C80ED11C84EEC81685E0CB
:1021B000D80669F70E94830F80914A0500FB87F9D2
:1021C00080934A05902F969580914B058078892BB6
:1021D00010FB87F980934B05E0924C05F0924D057A
:1021E000552051F060914A0570914B0580914C0546
:1021F00090914D050E94A80F0F900F900F90DF91C6
:10220000CF911F910F91FF90EF90DF90CF90BF90F3
:10221000AF909F908F907F906F905F900895CF9335
:1022200090914A0590FF41C09178811102C092605F
:1022300007C0833210F0946403C08F73880F982B0B
:1022400090934A05662351F060914A0570914B05C1
:1022500080914C0590914D050E94A80FC0914A05B0
:102260006C2F66956F7370E04BE050E081E394E073
:102270000E947732892B19F010924F0503C081E03C
:1022800080934F05CC1FCC27CC1F90914B05892FF5
:10229000880F97FB992790F920E040914D056091B8
:1022A0004C058C2BCF910C944A10CF91089561E08E
:1022B0000C940F1180914A0586958F73815009F413
:1022C00082E261E00C940F1180914A0586958F732C
:1022D0008F5F833208F081E061E00C940F11CF939F
:1022E000DF9300D01F92CDB7DEB720914A0520FFC3
:1022F0001AC09E012F5F3F4F0E94D60F2B8139815C
:102300004A8180914A0580FF0EC080E090E0FC0188
:10231000EE52FA4F41833083228303968231910536
:10232000B1F70E94830F0F900F900F90DF91CF9124
:10233000089581E080939D0468E070E081EF93E070
:102340000C94AC2581E080939E0468E070E081E706
:1023500093E00E94AC2568E070E081E393E00C9488
:10236000AC256091FE0561606093FE0587E090E01A
:102370000E949B2D62E070E081E193E00C94AC251B
:102380001F920F920FB60F9211244F925F926F928D
:102390007F928F929F92AF92BF92CF92DF92EF92F5
:1023A000FF922F933F934F935F936F937F938F93FE
:1023B0009F93AF93BF93CF93DF93EF93FF9380915E
:1023C000FD05882309F4C2C1C091FC04D091FD042D
:1023D0001C161D060CF0BAC14090F8045090F90488
:1023E0006090FA047090FB0420E030E0A901C30182
:1023F000B2010E94583018160CF065C0C130D105EA
:1024000009F452C08091F6049091F704BE010E9435
:102410005D327C019093F7048093F6048090F3057D
:102420009090F405A090F505B090F60520E030E01E
:1024300040E85FE3C501B4010E94332E6093F305C9
:102440007093F4058093F5059093F605F701EE0F70
:10245000FF1FEE0FFF1FEA52FB4FA30192016081A5
:102460007181828193810E94A42E20E030E040E0BF
:102470005EE30E94D3309B01AC01C501B4010E9410
:10248000583018168CF4C7010196BE010E945D32C7
:102490009093F7048093F6041092F3051092F405DC
:1024A0001092F5051092F605E091F604F091F7040C
:1024B000EE0FFF1FEE0FFF1FEA52FB4FC080D180CF
:1024C000E280F380E0C0809110032197882309F413
:1024D000BFC0C090D204D090D304E090D404F09058
:1024E000D50420E030E0A901C701B6010E949F2E6B
:1024F000882309F4A2C0FE01EE0FFF1FEE0FFF1F9D
:10250000EA52FB4F80809180A280B380A5019401A4
:10251000C701B6010E949F2E87FF31C0A50194011B
:1025200060E070E08CED93EC0E94A42E20E030E09F
:1025300040E451E40E94A42E20E030E040E05FE35C
:102540000E94D3309B01AC0160E070E080E090E439
:102550000E9440319B01AC01C501B4010E94D330FF
:102560009B01AC01C701B6010E949F2E87FF07C0E7
:10257000A701960160E070E08CED93E439C0A501FD
:102580009401C701B6010E94583018160CF055C0CE
:10259000A501940160E070E08CED93E40E94A42E0C
:1025A00020E030E040E451E40E94A42E20E030E03E
:1025B00040E05FE30E94D3309B01AC0160E070E03B
:1025C00080E090E40E9440319B01AC01C501B40160
:1025D0000E94D3309B01AC01C701B6010E94583064
:1025E00018165CF5A701960160E070E08CED93ECA5
:1025F0000E94A42E20E030E040E451E40E94A42E8A
:1026000020E030E040E05FE30E94D3309B01AC016A
:1026100060E070E080E090E40E9440319B01AC01FA
:10262000C701B6010E94D3306093D2047093D304E3
:102630008093D4049093D5041EC0CC0FDD1FCC0F23
:10264000DD1FCA52DB4F88819981AA81BB810BC0F3
:10265000FE01EE0FFF1FEE0FFF1FEA52FB4F8081BE
:102660009181A281B3818093D2049093D304A093EB
:10267000D404B093D504C090D204D090D304E09099
:10268000D404F090D5048091D0049091D1048F3F70
:102690002FEF920729F001969093D1048093D004F4
:1026A00080918504811116C01092100380E090E0A3
:1026B000A0E0BFE380930C0390930D03A0930E035F
:1026C000B0930F031092F8041092F9041092FA04D8
:1026D0001092FB0420E034E244EF51E4C701B6015C
:1026E0000E949F2E87FF08C086EFC82E88E2D82E52
:1026F00084EFE82E81E4F82E20E030E040E051E461
:10270000C701B6010E94D3309B01AC0160E074E2C6
:1027100084E79BE40E94A42E6B017C010E94502F51
:10272000709387006093860020910C0330910D0315
:1027300040910E0350910F03C701B6010E94D330A0
:102740000E94502F70938900609388008091FC054F
:10275000882309F449C1C090EE05D090EF05E090C0
:10276000F005F090F10520E030E0A901C701B601C5
:102770000E94583018160CF052C08091D0049091ED
:10278000D1048F3F2FEF920729F001969093D10447
:102790008093D00480918504811116C0109210039B
:1027A00080E090E0A0E0BFE380930C0390930D03E2
:1027B000A0930E03B0930F031092F8041092F90443
:1027C0001092FA041092FB0420E030E040E051E463
:1027D000C701B6010E94D3309B01AC0160E074E2F6
:1027E00084E79BE40E94A42E6B017C010E94502F81
:1027F000709387006093860020910C0330910D0345
:1028000040910E0350910F03C701B6010E94D330CF
:102810000E94502F709389006093880008C0109226
:1028200087001092860010928900109288006091B3
:10283000E8057091E9056F5F7F4F7093E90560933C
:10284000E805209186003091870080E090E0232BFE
:1028500071F12091CF0421112AC0C0918600D0913E
:1028600087000E947F2F6B017C01BE0180E090E019
:102870000E947F2F9B01AC016091EA057091EB05EE
:102880008091EC059091ED050E94A42E20E03FEF91
:102890004FE757E40E94D33020E030E040E85FE3A8
:1028A0000E94322E9B01AC01C701B6010AC00E94F2
:1028B0007F2F2091EA053091EB054091EC05509176
:1028C000ED050E94583087FD8FC08091F2058F5F23
:1028D0008093F20590E02091F8053091F905821778
:1028E0009307A0F08091F705882319F01092F20564
:1028F0000DC080916F008D7F80936F00809180006C
:102900008F73809380001092FC0576C09091CF0465
:102910008091F205E091FA05F091FB05911137C025
:1029200091E09093CF0481508093F20598E0899FC5
:10293000E00DF11D1124C080D180E280F38020855C
:10294000318542855385C701B6010E949F2E8111B2
:1029500009C01092EE051092EF051092F00510924A
:10296000F10508C0C092EE05D092EF05E092F005A7
:10297000F092F10580E090E0A0E8BFE38093EA05E3
:102980009093EB05A093EC05B093ED0529C0109250
:10299000CF041092D1041092D00428E0829FE00D61
:1029A000F11D112480819181A281B3818093EE0574
:1029B0009093EF05A093F005B093F10520E030E08F
:1029C00040E85EE364817581868197810E94D330FF
:1029D0006093EA057093EB058093EC059093ED0509
:1029E0001092E9051092E8058091FE0580FD04C073
:1029F0001092FC051092FD05FF91EF91DF91CF91B0
:102A0000BF91AF919F918F917F916F915F914F9106
:102A10003F912F91FF90EF90DF90CF90BF90AF90BC
:102A20009F908F907F906F905F904F900F900FBE10
:102A30000F901F9018950E94C821811102C00E941A
:102A4000D32187E090E00E94872D8093FE0580913E
:102A5000FF05811129C0259A80916F008D7F809399
:102A60006F0082E0809380008AE18093810081EC96
:102A700091E1909387008093860023EA3BE04EE843
:102A800055E460910C0370910D0380910E039091B9
:102A90000F030E94D3300E94502F709389006093DF
:102AA000880081E08093FF058091FE0580FF06C0CD
:102AB00063E070E084EF92E00C94AC25089580917F
:102AC000FF05811102C00E941B151092FD04109297
:102AD000FC0480916F008D7F80936F008091800057
:102AE0008F73809380001092FC051092FD05109268
:102AF000D2041092D3041092D4041092D5041092F0
:102B0000CB041092CC041092CD041092CE041092FB
:102B1000CA041092C904E6EDF4E0A9EBB4E0119206
:102B20001192119211921D921D9284E0E63FF807D6
:102B3000B1F7089580919E0481110C945F1508955A
:102B40000E949A1510929E0468E070E081EB93E079
:102B50000C94AC2562E070E081E293E00E94AC2529
:102B60002FEF81EE94E0215080409040E1F700C0CB
:102B700000000E945F156091FE056E7F6093FE0568
:102B800087E090E00C949B2DAF92BF92CF92DF92A2
:102B9000EF92FF920F931F93CF93DF9300D000D05B
:102BA000CDB7DEB7682F70E065547109072E000CB1
:102BB000880B990B0E94812F20E030E040E451E423
:102BC0000E94A42E9B01AC0160E070E080E090E4E4
:102BD0000E9440312091FD05222309F4A1C02091DB
:102BE000FF0521110AC069837A838B839C830E942D
:102BF0001B159C818B817A81698120E030E04CED4E
:102C000053E40E94D3306B017C0106EF14E027E00F
:102C1000A22EB12CA7019601F80192918291729196
:102C200062918F010E949F2E811134C0F501EE0F39
:102C3000FF1FEE0FFF1FEA52FB4F1082118212821C
:102C40001382D501AA0FBB1FA754BB4F11961C922C
:102C50001E9287E0A816B10411F18FEFA81AB80AE6
:102C60004481558166817781408351836283738378
:102C7000148215821682178212968D919C91139759
:102C800011969C938E9313961C921E9212973496D3
:102C90001296DFCFE1E0AE1AB10808F0BBCF809109
:102CA000FC049091FD04019797FD05C09093FD04ED
:102CB0008093FC0404C01092FD041092FC048091E7
:102CC000FC049091FD042091F6043091F70428173C
:102CD000390724F01092F7041092F604892B01F5BD
:102CE00080916F008D7F80936F00809180008F7343
:102CF000809380001092D2041092D3041092D404D6
:102D00001092D5041092CB041092CC041092CD04F2
:102D10001092CE041092CA041092C9041092FD05BC
:102D20000F900F900F900F90DF91CF911F910F9107
:102D3000FF90EF90DF90CF90BF90AF900895CF922B
:102D4000DF92EF92FF92CF93DF9300D000D0CDB708
:102D5000DEB7682F70E065547109072E000C880BF0
:102D6000990B0E94812F20E030E040E451E40E9462
:102D7000A42E9B01AC0160E070E080E090E40E9432
:102D800040312091FF0521110AC069837A838B832A
:102D90009C830E941B159C818B817A816981209183
:102DA000FE0520FF5AC02091FC043091FD0428301C
:102DB00031050CF052C020916F002D7F20936F00E1
:102DC0002091FC05222351F069837A838B839C83B5
:102DD0000E945F159C818B817A81698120E030E0BF
:102DE0004CED53E40E94D3306B017C0181E0809371
:102DF000FD051092D1041092D00420E030E0A9012A
:102E0000C701B6010E9458301816ECF48091FC04FA
:102E10009091FD04FC01EE0FFF1FEE0FFF1FEA5221
:102E2000FB4FC082D182E282F382FC01EE0FFF1FD2
:102E3000E754FB4F2FE030E03183208301969093DD
:102E4000FD048093FC0480916F00826080936F008A
:102E5000809180008068809380000F900F900F9089
:102E60000F90DF91CF91FF90EF90DF90CF9008957A
:102E7000CF9380919A04882309F441C080919604ED
:102E800090919704009781F40E9479219093970480
:102E9000809396042091980430E02115310571F457
:102EA0008091990490E00BC00E944F212091A902CB
:102EB0003091AA022817390738F321C0C9010197B8
:102EC000FC01EA57FB4F8081F901EA57FB4FC081B3
:102ED00090919E0491110E94C41580919E048823B4
:102EE00019F08C2F0E949F168091980490E0019613
:102EF0006091990470E00E945D3280939804CF91B4
:102F00000895CF93DF9327E0729FF001112438E3F7
:102F1000839FE00DF11D1124E60FF11DEE0FFF1F41
:102F2000EE51FE4FC591D491CE01C238D10549F181
:102F3000B0F4C133D10509F464C048F4C932D105F5
:102F400009F458C0CA32D10509F462C068C0C5335B
:102F5000D10509F448C0C933D10599F060C0C33E1A
:102F6000D10541F138F4C03ED10591F0C23ED10502
:102F7000B1F055C0C63ED10521F1C73ED10561F182
:102F80004EC020911E0520FD06C221FD04C205C2CF
:102F900020911E0520FF01C289E390E0FEC120912F
:102FA0001E0522FFFAC180911E0584FDA6C183EE95
:102FB00090E0F3C180911E0582FFF5CF82EE90E094
:102FC000ECC120911E0523FFE8C180911E0584FD00
:102FD00094C187EE90E0E1C180911E0583FFF5CF9B
:102FE00086EE90E0DAC120911E0525FFD6C189E268
:102FF00090E0D3C120911E0525FFCFC185E390E06D
:10300000CCC120911E0526FFC8C18AE290E0C5C14F
:1030100020911E0526FFC1C181E390E0BEC1C1150C
:1030200040E5D40708F049C0C11550E4D50708F0C1
:1030300032C1C83ED10520F5C03ED10508F0ADC172
:10304000C83AD10570F4C53AD10508F0AEC0C13018
:10305000D10509F4A2C108F450C1249708F44DC168
:103060009CC1CF3BD10508F4ABC0C03CD10508F4EE
:1030700044C1CE01880F991F825F9B4FFC01FFC0A6
:10308000C11520E2D20760F4C11531E0D30708F082
:1030900084C1C03FD10508F430C1CE0190657DC127
:1030A000C11540E3D40708F0EDC0CE019F70FC01CC
:1030B000EE0FFF1FE257FA4FE2C0C11555E5D507E5
:1030C00008F046C0C11584E5D80708F0FCC0C1155A
:1030D00092E5D90720F5C11521E5D20708F0DFC038
:1030E0002C2F237081E090E002C0880F991F2A9551
:1030F000E2F79C689E01F4E036952795FA95E1F792
:103100002370FC01F22B8C2F8F70982F969596953B
:1031100030E2939FC00111248E2B9F2B3EC18C2F38
:1031200086958695AE0143705527C115D34508F0A5
:10313000BBC090E2899F9001112481E090E002C021
:10314000880F991F4A95E2F7822B932B9C6825C123
:10315000C11549E5D40798F4C11558E5D50708F01D
:10316000B7C0C11586E5D80708F0C7C08C2F0E94EC
:103170003A0E8F7190E0982F882790620EC1C1158A
:103180009AE5D90708F4A9C0CE019056811590425E
:1031900008F0B3C08D2F8F710E943A0EDD27D062E8
:1031A0008F719E01382BC901F8C0C53AD10509F4C9
:1031B000A7C0C63AD10509F0A6C082E890E4EDC0E8
:1031C000C83AD10509F4A2C0C93AD10509F4A1C091
:1031D000CA3AD10509F4A0C0CB3AD10509F49FC081
:1031E000CC3AD10509F49EC0CB3BD10509F49DC072
:1031F000CC3BD10509F49CC0CD3AD10509F49BC064
:10320000C03BD10509F49AC0CE3AD10509F499C062
:10321000CF3AD10509F498C0C13BD10509F497C054
:10322000C23BD10509F496C0C33BD10509F495C052
:10323000C43BD10509F494C0C53BD10509F493C042
:10324000C63BD10509F492C0C73BD10509F491C032
:10325000C83BD10509F490C0C93BD10509F48FC022
:10326000CD3BD10509F48EC0CE3BD10509F48DC00C
:10327000CA3BD10509F48CC080E094E48EC08591EE
:1032800094918BC09E013327C901D3FF02C0986C73
:1032900084C0906C82C0CE019F70906A7EC09C2FCB
:1032A0008827816F906A79C090E2899F90011124EC
:1032B00081E090E002C0880F991F4A95E2F7822BC7
:1032C000932B9A686AC09C2F8827846F906A65C088
:1032D0009C2F8827806F906A60C02C2F2F70206EE3
:1032E00030E0306ACE0144E0969587954A95E1F743
:1032F0008F70A901582BCA0150C080E090E04DC0EA
:1033000081E890E44AC083E890E447C082EE94E408
:1033100044C089EE94E441C08AEE94E43EC085EB5B
:1033200094E43BC086EB94E438C083EB94E435C06E
:1033300084EB94E432C087EB94E42FC08CEC94E4EB
:103340002CC08DEC94E429C083E895E426C08AE87B
:1033500095E423C082E995E420C084E995E41DC08A
:1033600081E296E41AC083E296E417C084E296E410
:1033700014C085E296E411C086E296E40EC087E2AE
:1033800096E40BC08FE694E408C080E794E405C09F
:103390008AE296E402C080EE90E0DF91CF9108953A
:1033A0001F93CF93DF93EC01FE012491222309F4B4
:1033B00034C0CE010196213021F4EC01FC011491BE
:1033C00024C0223031F4EC01FC0184910E94632C72
:1033D00022C0233021F4EC01FC0184911AC030E0BA
:1033E000F901E25FFA4F1491F901E257FB4F249182
:1033F000222359F081EE0E94632C812F0E94632CBE
:10340000812F0E942B2C81EE04C0812F0E94632CFF
:10341000812F0E942B2C2196C7CFDF91CF911F9136
:103420000895CF93DF93EC01682F83E090E00E9432
:103430009B2DBE0180E090E0DF91CF910C9455234D
:10344000E8EDF0E08081806180838AE18A95F1F780
:1034500000C08091D90081700895A5E7B4E041E0F3
:1034600050E08D91E82FE295EF70F0E021A18F7090
:10347000BA0102C0660F771F8A95E2F7CB01962F3B
:103480009095922391A392A1892B82A374E0A937EE
:10349000B70739F708959F92AF92BF92CF92DF920C
:1034A000EF92FF920F931F93CF93DF9380913C0491
:1034B000811103C004E010E002C000E010E0A801A8
:1034C0004A5E5A4F7A01EA0185E7C82E84E0D82E79
:1034D000AA24A394B12C25E0922E89E7C81684E093
:1034E000D80609F448C0F60181916F01E82FE295F2
:1034F000EF70F0E021A18F70A50102C0440F551FAD
:103500008A95E2F7CA01922F982B91A392A18095F8
:10351000892382A350EA5A95F1F7EDE7F4E020E021
:1035200040E050E03191A32FA295AF70B0E09096AB
:103530008C9190E03F7002C0959587953A95E2F79F
:1035400080FD07C0C501042E01C0880F0A94EAF768
:1035500002C080E090E0282B4F5F5F4F473051055D
:1035600009F78881821719F028839092F3020E944C
:103570002D1A2196B2CF8091F3028823E1F0815079
:103580008093F302882339F0EFE9FFE03197F1F7F8
:1035900000C0000010C080E090E0FC01E00FF11FCF
:1035A000ED5DFA4FD701A80FB91F2C91208301962A
:1035B0008430910591F781E0DF91CF911F910F91B8
:1035C000FF90EF90DF90CF90BF90AF909F900895C5
:1035D0000F931F93CF93DF9380911505882309F4F0
:1035E00074C00E944B1A80913C04811103C0E4E036
:1035F000F0E002C0E0E0F0E0ED5DFA4F80E090E046
:103600002191DC01AA5FBA4F2C9301968430910579
:10361000B9F780913C04811103C000E010E002C0C2
:1036200004E010E0C0911105D0911205F894529A6F
:103630005A9885E08A95F1F7000052985A9A80E2EC
:103640008A95F1F74A9B08C0529A5A9AE881F98103
:1036500081E0808378946CC06D81662379F08E81DF
:103660009F810E946B0E811109C0529A5A9AE8817B
:10367000F98182E08083789428985AC00E945D0E78
:1036800080E28A95F1F75A98529A80E18A95F1F78B
:103690006A81662321F08B819C810E94920E0E9498
:1036A000650EE881F98110827894289AF801ED5D21
:1036B000FA4F80E090E0DC01AE5FBA4F2C9121938D
:1036C000019684309105B9F72FC00E944B1A809162
:1036D0003C04811103C0E4E0F0E002C0E0E0F0E06F
:1036E000ED5DFA4F80E090E02191DC01AE5FBA4FD2
:1036F0002C93019684309105B9F780913C04811197
:1037000003C0E0E0F0E002C0E4E0F0E0ED5DFA4F7D
:1037100080E090E0DC01AA5FBA4F2C9121930196E2
:1037200084309105B9F71BC05D9A1092B80417C098
:103730005D988091B8048F5F8093B804863078F0EC
:1037400080913C04811103C0E0E0F0E002C0E4E0BD
:10375000F0E0ED5DFA4F10821182128213820E9416
:10376000381781E0DF91CF911F910F9108951F923B
:103770000F920FB60F9211242F933F934F935F93A5
:103780006F937F938F939F93AF93BF93CF93DF9369
:10379000EF93FF935A98529AC0911105D091120558
:1037A0006D81662321F08E819F810E94920E0E947E
:1037B000650E80E18A95F1F75A9852985A9A80E1FD
:1037C0008A95F1F76A81662351F08B819C810E9472
:1037D0006B0EE881F981811104C082E003C0E881A9
:1037E000F98188E080830E945D0EFF91EF91DF9167
:1037F000CF91BF91AF919F918F917F916F915F9189
:103800004F913F912F910F900FBE0F901F901895E1
:103810001F920F920FB60F9211248F939F93EF93E5
:10382000FF938091B900887F803869F038F488234D
:10383000C9F18036C9F51092B70436C0883A09F14B
:10384000883BF9F031C08091B704811111C080919B
:10385000BB008093B6048091B604803120F01092B2
:10386000B60480E001C081E091E09093B7041DC0F0
:10387000E091B604F0E08091BB00EA55FB4F8083F5
:1038800008C0E091B604F0E0EA55FB4F80818093D8
:10389000BB008091B60490E001968F7099278093C9
:1038A000B60402C01092BC0081E09091BC00956803
:1038B0008295880F880F807C892B8093BC00FF91B4
:1038C000EF919F918F910F900FBE0F901F901895C1
:1038D00008958091BD050895CF93DF9300D01F9286
:1038E000CDB7DEB79C0190910F05911105C0809175
:1038F000C805843049F504C0923011F0943021F5A8
:1039000084E089833B832A8382E08093E9008FEF00
:103910009091E800815095FD06C095ED9A95F1F7DC
:1039200000008111F5CF8091E80085FF0DC040E0D7
:1039300050E063E070E0CE0101960E944426809141
:10394000E8008E778093E8000F900F900F90DF9142
:10395000CF910895CF93DF9300D01F92CDB7DEB7FC
:103960002091C805243031F523E02983805891093E
:103970009B838A8382E08093E9008FEF9091E80037
:10398000815095FD06C095ED9A95F1F700008111E3
:10399000F5CF8091E80085FF0DC040E050E063E086
:1039A00070E0CE0101960E9444268091E8008E7757
:1039B0008093E8000F900F900F90DF91CF910895C2
:1039C000CF93DF9320910F05211103C02091C805EB
:1039D00002C0223011F0243039F521E02093E900B3
:1039E0002FEF3091E800215035FD06C035ED3A95B6
:1039F000F1F700002111F5CF2091E80025FF14C058
:103A0000EC0140E050E068E070E00E9444268091C4
:103A1000E8008E778093E80088E0FE01AEEBB5E029
:103A200001900D928A95E1F7DF91CF910895CF93A0
:103A3000DF93CDB7DEB72A970FB6F894DEBF0FBE7F
:103A4000CDBF84B7877F84BF0FB6F894A8958091C7
:103A50006000886180936000109260000FBE80E873
:103A6000809361001092610085B7806885BF85B73B
:103A7000806885BF0E94201A80933C040E94201A0F
:103A8000882361F08DE394E09093120580931105F3
:103A900081E080931005529A5A9A11C08DE394E008
:103AA000909312058093110581E080931005529840
:103AB0005A9AEA9A809169008F7C80936900789481
:103AC0000E9494290E94392A8091E20084608093A8
:103AD000E20078948091C8058823A1F01091E90054
:103AE0001F709091EC00892F817090FD80E8182B59
:103AF0001092E9008091E80083FD0E947B261F70F0
:103B00001093E90082E084BD93E095BD9AEF97BDE4
:103B100080936E0080912C058360886080932C05D3
:103B20000E942D1AADE7B4E041E050E08D91E82FFE
:103B3000E295EF70F0E021A18F70BA0102C0660F2C
:103B4000771F8A95E2F7CB01962F9095922391A348
:103B500092A1892B82A374E0A438B70739F7559A4C
:103B6000209A5D9A289AA6E1B5E0E3E2F5E038E014
:103B7000532E5E0E11921D925E12FCCF0E94201AEF
:103B8000809315050E94C821811102C00E94D32193
:103B90000E941B158FEF90E7E2E081509040E040DB
:103BA000E1F700C0000080914A0586958F7390E090
:103BB00090931405809313050E94C821811102C0BF
:103BC0000E94D32182E090E00E94872D80932C05F3
:103BD00084E090E00E94872D90E090931F058093F1
:103BE0001E0583E090E00E94872D682F70E080E042
:103BF00090E00E94552380912C05816080932C05D4
:103C00000E94C821811104C00E94D3210E94C60FC6
:103C100088E090E00E948F2D60934A0570934B05D9
:103C200080934C0590934D056E7771F40E94C60FFA
:103C300088E090E00E948F2D60934A0570934B05B9
:103C400080934C0590934D0581E080934F058091C2
:103C50004A0580FF05C0869560E08F730E940F11B2
:103C600087E494E0909321058093200588E7482E0F
:103C700096E0A92EB12C28E6C22EDD24D3948091A3
:103C8000C805853009F037C08091C805843021F11E
:103C90001092220520E488E190E00FB6F894A895F0
:103CA000809360000FBE2093600083B7817F8460A3
:103CB00083BF83B7816083BF7894889583B78E7FF5
:103CC00083BF0FB6F894A8958091600088618093B7
:103CD0006000109260000FBE8091C705882309F430
:103CE000CECF0E94E81AE3E2F5E0819181119BC2F8
:103CF0005E12FBCFC4CF0E94E81AADE2B5E0E3E26A
:103D0000F5E000E010E0702F61912D912627C1F1C0
:103D100080E090E030E0F82EA901082E02C0559511
:103D200047950A94E2F740FF27C089837A8381E0B0
:103D300090E09C0102C0220F331FFA94E2F7790150
:103D4000862F90E08223932321E0892B09F420E041
:103D50002B830E9479218160782F9D838C834981F8
:103D60005A816B818D810E94B40EF801E35DFA4F98
:103D70008081E826E0821AC001968730910559F6C5
:103D80000F5F1F4F0830110509F0BDCF8FEF8E83F5
:103D90008F8318860E9479218160782F9A8789877E
:103DA0004E815F8168858A850E94B40E10912B0533
:103DB0000E94770F181721F00E94770F80932B0530
:103DC00080914F05882309F45ACF80914A05182F16
:103DD00016951F739EE3910F9F73943008F055C0A2
:103DE00080913605909137050E944F21EEEFE10F4B
:103DF000F0E0E856F94FE491F0E08E179F0708F4E1
:103E00003ECF0E94792190933705809336056091CB
:103E1000350570E080E090E00E94812F20E030E0E6
:103E20004FE753E40E94A42E2BED3FE049E450E419
:103E30000E94D3300E9490310E941E2F2BE43AE35F
:103E40004EE25FE30E94322E20EF3BEF48ED52E45A
:103E50000E94D3300E94502F462F80914A05881F20
:103E60008827881F90914B05292F220F97FB9927B0
:103E700090F960914C05822B0E946F11809135055D
:103E800090E0019680933505FACE9AE3910F9F73E7
:103E9000933070F580913A0590913B050E944F2137
:103EA000EAEFE10FF0E0E456F94FE491F0E08E170D
:103EB0009F0708F4E4CE0E94792190933B058093FC
:103EC0003A0540914D0560914C05809138059091DF
:103ED00039050E946F11809138059091390501963E
:103EE000B6010E9449329093390580933805C7CEB8
:103EF00097E3910F9F73963008F04CC007EF902E18
:103F0000910E80913E0590913F050E944F21E92D31
:103F1000E695F0E0E156F94FE491F0E08E179F0747
:103F200008F4ADCE0E94792190933F0580933E0521
:103F3000B2EDEB2EB5E0FB2E00E010E080913C05E9
:103F400090913D05800F911FB6010E944932970163
:103F500040914D0560914C050E94D60F045C1F4FA7
:103F600033E0E30EF11C083661E0160739F70E94D2
:103F7000830F80913C0590913D0590FE05C0019610
:103F8000B8010E94493201C0019790933D0580938A
:103F90003C0575CE91E3910F9F73963008F082C077
:103FA0001F5010FF03C033243A9402C033243394CB
:103FB00080914105909142050E944F21E12FE695A5
:103FC000F0E0EE55F94FE491F0E08E179F0708F40A
:103FD00056CE0E9479219093420580934105F2EDDF
:103FE0008F2EF5E09F2EA4EDEA2EA5E0FA2E00E03C
:103FF00010E0F70131971082F4011082F70110826E
:10400000E4E06E2E712C212C80914005820D87FDFD
:104010008A5F082E000C990B08171907E9F48091A4
:104020004D05869DA001879D500D112455954795FE
:104030005595479580914A05881F8827881F90913C
:104040004B05592F550F97FB992790F994016091D3
:104050004C05852B0E94D60F230CF1E06F1A7108D6
:1040600099F60F5F1F4F23E0820E911C33E0E30EA1
:10407000F11C0630110509F0BCCF0E94830F80911E
:10408000400561E0361208C0811102C085E001C020
:10409000815080934005F3CD90E00196B8010E94D5
:1040A0005D32F7CF9BE2910F9F73933008F077C09A
:1040B00080914405909145050E944F21EBEEE10F60
:1040C000F0E0EB55F94FE491F0E08E179F0708F40C
:1040D000D6CD0E947921909345058093440580E0D8
:1040E00090E0FC01EE52FA4F118210821282039688
:1040F00082319105B1F700E010E0C801B5010E94DE
:104100005D3240914305042E000C550B9C01220F9B
:10411000331F820F931F04171507FCF040914604CC
:10412000042E000C550B40175107BCF09C012E5279
:104130003A4F80914A05881F8827881F90914B0528
:10414000592F550F97FB992790F940914D05609194
:104150004C05852B0E94D60F06C0FC01EE52FA4F8B
:104160001182108212820F5F1F4F0630110529F64F
:104170000E94830F8091450490914305980F90937E
:10418000430520914604280F2093460412161CF480
:1041900095300CF474CD81958093450470CD8E7765
:1041A000803309F06CCD80914805909149050E94BB
:1041B0004F21883E934008F462CD0E94792190936C
:1041C00049058093480500914605109147050F5F0A
:1041D0001F4F01701127109347050093460582ED8C
:1041E000882E85E0982EF12C8F2D8695F801E80F0A
:1041F000F11DCF0181709927940140914D05609187
:104200004C05FC014E9EC0014F9E900D11240E9452
:10421000D60FF394F3E08F0E911C26E0F212E4CF58
:104220000E94830F2CCD80E189BD82E189BD09B454
:1042300000FEFDCF8091D8008F7D8093D8008091C3
:10424000E00082608093E0008091E00081FDFCCF7F
:1042500016CD78941F920F920FB60F9211248F9360
:104260009F93AF93BF9380910B0590910C05A09104
:104270000D05B0910E050196A11DB11D80930B0592
:1042800090930C05A0930D05B0930E05BF91AF91CF
:104290009F918F910F900FBE0F901F901895CF9206
:1042A000DF92EF92FF920F931F932FB7F8944091F4
:1042B0000B0550910C0560910D0570910E052FBFF7
:1042C0006A017B01EE24FF248C0120E030E0C0165F
:1042D000D106E206F30610F4415051099A01281B59
:1042E000390BC9011F910F91FF90EF90DF90CF9094
:1042F00008952FB7F89480910B0590910C05A0912B
:104300000D05B0910E052FBF08951F920F920FB6A5
:104310000F9211248F939F93AF93BF9380912205A7
:10432000811113C080910B0590910C05A0910D0592
:10433000B0910E054196A11DB11D80930B05909380
:104340000C05A0930D05B0930E05BF91AF919F9101
:104350008F910F900FBE0F901F9018959C01FC013C
:1043600032969FEF80E04191461789F09F3F19F404
:10437000411101C0982F8F5F8630A9F79F3F39F018
:10438000F901E90FF11D97FDFA95628308950895EB
:1043900080E090E00E94952D21E08D3E9E4F09F037
:1043A00020E0822F08956DEE7EEF80E090E00E9485
:1043B000B92D60E082E090E00E949B2D60E083E0F8
:1043C00090E00E949B2D1092B7051092B8051092B4
:1043D000B9051092BA0560E084E090E00E949B2D40
:1043E00060E085E090E00E949B2D60E086E090E038
:1043F0000E949B2D6FEF87E090E00E949B2D40E094
:1044000050E0BA0188E090E00E94AD2D60E08DE0C0
:1044100090E00E949B2D40E050E0BA018FE090E0D8
:104420000E94AD2D40E050E0BA0183E190E00C9491
:10443000AD2D9091B6058091BB05892B2091B505D6
:10444000982F922B909350058091B405882391F07A
:10445000892B80935005E2E5F5E080E096E09E0F21
:104460009E1729F021912223D9F38F5FF9CF811173
:104470001092B405E0912005F0912105309731F0BC
:104480000280F381E02D80E595E009940895BF92C4
:10449000CF92DF92EF92FF920F931F93CF93DF9310
:1044A0008C01C090B705D090B805E090B905F090A8
:1044B000BA058091E4059091E505A091E605B091DB
:1044C000E705C82AD92AEA2AFB2ACFE1D0E0D7019A
:1044D000C6010C2E04C0B695A795979587950A94AA
:1044E000D2F780FF07C0BC2EB8018C2F0E94811725
:1044F000019719F4219758F7B12C8B2DDF91CF91AB
:104500001F910F91FF90EF90DF90CF90BF90089593
:10451000CF93DF93EC010E944722BE010E948117D6
:10452000DF91CF91089527E0929F800D1124682F8D
:10453000669566956695982F977085E0689FB0019F
:10454000112440E050E080E0FA01E60FF71FE05749
:10455000FA4F208130E0092E02C0369527950A9443
:10456000E2F721703327042E01C0220F0A94EAF7E4
:10457000822B4F5F5F4F4530510531F7089527E09B
:10458000929F800D1124A82FA695A695A6958770B9
:1045900051E001C0550F8A95EAF785E0A89FD00148
:1045A000112420E030E070E0F901EA0FFB1FE05732
:1045B000FA4F4081CB01022E02C0969587950A944E
:1045C000E2F781709927819584278523842780834A
:1045D0002F5F3F4F2530310539F708956093E4058B
:1045E0007093E5058093E6059093E7050C94FF2B07
:1045F0000F931F9341E050E060E070E004C0440F6F
:10460000551F661F771F8A95D2F740955095609584
:1046100070958091E4059091E505A091E605B09133
:10462000E7058A019B01082319232A233B23C9019B
:10463000B8011F910F910C94EE222091B305809543
:1046400082238093B305982F977069F430E0482F48
:10465000082E000C550B2417350729F085958595F4
:1046600085950C94F82208950F931F9341E050E034
:1046700060E070E004C0440F551F661F771F8A95E5
:10468000D2F78091E4059091E505A091E605B091FF
:10469000E7058A019B01082B192B2A2B3B2BC9010B
:1046A000B8011F910F910C94EE226093B70570939F
:1046B000B8058093B9059093BA050C94FF2B8091AF
:1046C0008F0590915E05891719F08F5F8770FBCF7A
:1046D000089580915D0582958F7009F054C0809196
:1046E0005A05882309F44FC080918F05A0915E057B
:1046F000609158057091590540915B0550915C059A
:10470000B6E08A1709F43FC090E041155105C1F1A8
:104710007F3F11F46F3FA1F1B89FF001B99FF00DF9
:104720001124E15AFA4F218172132AC020816213A9
:1047300027C02281211124C0238134812417350709
:1047400010F421503109241B350B24363105C0F4F7
:1047500020915D052F70206120935D0526E0289F44
:10476000F001299FF00D1124EC59FA4F80818F70D0
:104770008061808388E595E00E941A040C945F2391
:1047800001968770BECF0895BF92CF92DF92EF92CD
:10479000FF920F931F93CF93DF93CDB7DEB761974F
:1047A0000FB6F894DEBF0FBECDBF7C0185E0F701E8
:1047B000DE011D9601900D928A95E1F7D7013C919B
:1047C00011962C91119712960C9112971396CD90E9
:1047D000DC901497509158056091590580915B05C4
:1047E00090915C05009709F434C16F3F19F45F3F65
:1047F00009F42FC1B0905A05BB2009F4EDC04091D7
:104800005D05C816D90628F0F601E81BF90BCF01A3
:1048100004C0809590958C0D9D1D11E08436910506
:1048200048F010E0407F09F0A1C088E595E00E94C3
:104830001A0407C1842F807F09F044C0621312C09C
:10484000531310C001110EC04F70406140935D05BD
:1048500088E595E00E941A0480915D05D7011596C0
:104860008C932EC0CD2819F12F3F11F43F3FF9F062
:10487000102F01111CC080918F0540915E0556E0FC
:10488000841709F45AC090E0589FF001599FF00D29
:104890001124E15AFA4F6181261306C06081361354
:1048A00003C06281611103C001968770E9CF102FA8
:1048B000002309F4FBC080915D05816080935D0554
:1048C00010E0F4C062130DC053130BC0011109C0F6
:1048D00080915D05D70115968C93C7010E941A043B
:1048E00096C03D872E878D859E850E94D82B882374
:1048F000C9F10023B9F120915D05822F82958F7057
:1049000090E0029774F0809158059091590598872E
:104910008F831986DB86CA862C87CE0107960E9474
:104920001A0486E0F701A8E5B5E001900D928A959A
:10493000E1F70E94692311E0B9C03D872E878D857C
:104940009E850E948822292F22952F7030E02230E8
:1049500031050CF09FC09F7009F099C0805E8830CF
:1049600008F4A4C0C7010E941A04E5CF621314C062
:10497000531312C0011110C080915D05F7018583AA
:10498000C7010E941A0486E0E8E5F5E0DF011D9208
:104990008A95E9F71B2D8AC03D872E878D859E85D8
:1049A0000E94D82B8823F1F20023E1F220915D05CB
:1049B000822F82958F7090E002970CF4B2CF809195
:1049C0005805909159059A8389831B82DD82CC8298
:1049D0002E83CE010196A3CFC816D90638F0C81A87
:1049E000D90AB4E6CB16D10450F007C08095909553
:1049F0008C0D9D1D8436910510F010E022C0102F03
:104A0000002309F4AFCF62130BC0531309C086E033
:104A1000F701A8E5B5E001900D928A95E1F746C04F
:104A20003D872E878D859E850E94D82B811179CF59
:104A300080915D05816080935D05C7010E941A0425
:104A400035C0E8E5F5E086E0DF011D928A95E9F7DB
:104A50002DC0002309F486CF3D872E878D859E8546
:104A60000E94D82B182F882309F47CCF86E0F70109
:104A7000A8E5B5E001900D928A95E1F7809158057F
:104A8000909159050E9488220E9469230FC08111CC
:104A900065CF0CC0243031050CF064CF9F7009F451
:104AA0005DCFF7019581907F09F058CF812F6196F6
:104AB0000FB6F894DEBF0FBECDBFDF91CF911F912F
:104AC0000F91FF90EF90DF90CF90BF900895FC0181
:104AD0004AE04A95F1F798E030E080E021E040E1DB
:104AE0004A95F1F7880F4A9B02C08160322700C0C7
:104AF000000040E14A95F1F7915089F790E19A95CD
:104B0000F1F729B100C0000040E14A95F1F722FB1E
:104B1000992790F993272081920F9083089528E098
:104B200030E090E040E851E0642F682319F05A9A91
:104B3000952701C05A9860E26A95F1F74695215091
:104B4000310991F7992311F05A9A01C05A9880E2DD
:104B50008A95F1F75A9808950F931F93CF93DF9397
:104B6000EC018B018091FF05811102C00E941B1591
:104B70008091FE0580FF4DC080916F008D7F8093F6
:104B80006F008091FD0581110E945F1581E0809387
:104B9000FC05D093FB05C093FA051093F90500932B
:104BA000F8051092F7051092F3051092F405109293
:104BB000F5051092F6051092F20588819981AA8177
:104BC000BB818093EE059093EF05A093F005B09321
:104BD000F10520E030E040E85EE36C817D818E816C
:104BE0009F810E94D3306093EA057093EB05809318
:104BF000EC059093ED051092E9051092E80580917F
:104C00006F00826080936F00809180008068809345
:104C10008000DF91CF911F910F9108958091E4055D
:104C20009091E505A091E605B091E7058871992777
:104C3000AA27BB274897A105B10519F485E00C9474
:104C4000342385E00C94F8222BB1277F3BB13860E8
:104C50004FB7F894E2EDF5E08E529A4FE817F90756
:104C600089F0519168E03BB9000000C057FF2BB9B3
:104C7000550F000000C000C000C02BB900C06A95ED
:104C800091F7ECCF4FBF0895CF92DF92FF920F9331
:104C90001F93CF93DF931F92CDB7DEB7F82E8B0112
:104CA00099830E94B329998181111CC0CF2CD92EE0
:104CB00001151105B1F08091E80085FD0AC08091D1
:104CC000E8008E778093E8000E94B329882381F35F
:104CD00009C0F60181916F018093F1000150110923
:104CE000E7CF80E00F90DF91CF911F910F91FF9060
:104CF000DF90CF9008951F93CF93DF93CDB7DEB7AA
:104D0000AA970FB6F894DEBF0FBECDBFEAECF5E070
:104D100088E08E0F9091F10091938E13FBCF8091DC
:104D2000CB05833009F460C030F4813071F08230FB
:104D300009F49CC0B3C08A3009F488C08B3009F4F0
:104D40006BC0893009F0AAC020C08091CA05813AA1
:104D500009F0A4C08091E800877F8093E8008091EB
:104D6000CE059091CF05892B21F468E08EEB95E07C
:104D700003C060E080E090E070E00E94752B8091BD
:104D8000E8008B778093E80089C08091CA05813262
:104D900009F084C08091CE059091CF05029708F06C
:104DA0007DC08091E800877F8093E8008091E800D3
:104DB00082FD05C08091C8058111F8CF6FC0209198
:104DC000F3008091F20090E0922B029729F48091F9
:104DD000F1008B7F813021F48091F1008093BD053B
:104DE0008091E8008B7756C08091CA05813A09F01E
:104DF00055C08091CE059091CF05892B09F04EC00A
:104E00008091E800877F8093E8008091E80080FF30
:104E1000FCCF8091510439C08091CA058132F1F5EF
:104E20008091CE059091CF05892BC1F58091E80046
:104E3000877F8093E8000E94E5298091CC058093CC
:104E400051041092BB050E940D2C28C08091CA0508
:104E5000813221F58091E800877F8093E8000E94ED
:104E6000E5298091CD058093BC0518C08091CA05C5
:104E7000813AA1F48091E800877F8093E8008091D7
:104E8000E80080FFFCCF8091BC058093F100809109
:104E9000E8008E778093E8000E94E5298091E80081
:104EA00083FFD6C18091CA059091CB05492F50E070
:104EB0004A30510508F0CCC1FA01E757FF4F0C9476
:104EC0007132803821F0823809F0C2C108C0809167
:104ED000C6059091C705992389F082600FC0809123
:104EE000CE058F70873008F0B3C18093E9008091C0
:104EF000EB0085FB882780F91092E9009091E8008B
:104F0000977F9093E8008093F1001092F10074C1B4
:104F1000282F2D7F09F09CC1882319F0823061F081
:104F200097C18091CC05813009F092C1933009F08E
:104F300080E08093C7052EC08091CC0581112AC0E6
:104F40008091CE058F702FEF280F263008F080C19A
:104F50008093E9002091EB0020FF1CC0933021F4E6
:104F60008091EB00806214C09091EB00906190936F
:104F7000EB0021E030E0A90102C0440F551F8A95E3
:104F8000E2F74093EA001092EA008091EB0088601B
:104F90008093EB001092E9008091E800877F2FC199
:104FA000811156C11091CC051F778091E300807864
:104FB000812B8093E3008091E800877F8093E80055
:104FC0000E94E5298091E80080FFFCCF8091E300FA
:104FD00080688093E300111102C082E001C083E089
:104FE0008093C80535C18058823008F031C1809166
:104FF000CC059091CD058C3D53E0950779F583E084
:105000008A838AE289834FB7F894DE01139620E001
:105010003EE051E2E32FF0E050935700E49120FF8F
:1050200003C0E295EF703F5FEF708E2F90E0EA30A3
:1050300010F0C79601C0C0968D939D932F5F2431C9
:1050400049F74FBF8091E800877F8093E8006AE2CC
:1050500070E0CE0101960E94752BBDC04091CE0537
:105060005091CF05292F332723303105B9F06CF447
:105070002130310509F4FBC02230310509F0E8C0C8
:105080008BE390E0EEE1F7E054C02132310509F402
:1050900033C02232310509F43CC0DAC0992781308F
:1050A0009105D1F05CF4892B09F0D2C0EDE9F7E06D
:1050B000E4918E2F90E0EDE9F7E038C08230910561
:1050C00099F0039709F0C4C0EBE6F7E0E4918E2F66
:1050D00090E0EBE6F7E02AC0E7E8F7E0E4918E2FF6
:1050E00090E0E7E8F7E022C0E1E7F7E0E4918E2FF7
:1050F00090E0E1E7F7E01AC04115510509F4BCC0A2
:105100004130510509F0A4C089E090E0E9E4F7E0FE
:1051100010C04115510509F4B4C04130510509F0E2
:1051200097C086E390E0E8EAF6E003C0009709F450
:105130008FC02091E800277F2093E8002091D005C0
:105140003091D1052817390708F4C90140E00097CC
:1051500089F12091C805222309F43DC02530D9F1F9
:105160002091E80023FD37C02091E80022FD2FC0E8
:105170002091E80020FFEBCF4091F3002091F20056
:1051800030E0342B009759F02830310540F4449139
:105190004093F100319601972F5F3F4FF3CF41E0ED
:1051A0002830310509F040E02091E8002E77209367
:1051B000E800CDCF4111CDCF0AC08091C80588232A
:1051C00051F0853041F08091E80083FD04C080916A
:1051D000E80082FFF2CF8091E8008B778093E800AF
:1051E00037C08038A9F58091E800877F8093E80078
:1051F0008091C9058093F1008091E8008E778093BB
:10520000E8000E94E52924C0811122C01091CC053C
:105210001230F0F48091E800877F8093E8001093CB
:10522000C9050E94E529111106C08091E30087FDA0
:1052300002C081E001C084E08093C80542E061ECD7
:1052400081E00E94042A42E261EC82E00E94042A8A
:105250008091E80083FF1AC08091E800877F8093E7
:10526000E8008091EB0080628093EB000FC082E148
:1052700090E0E9E5F7E05DCF89E090E0E0E3F7E07A
:1052800058CF80E490E0EEEDF6E053CFAA960FB64B
:10529000F894DEBF0FBECDBFDF91CF911F9108956F
:1052A0001F920F920FB60F9211242F933F934F939B
:1052B0005F936F937F938F939F93AF93BF93CF939E
:1052C000DF93EF93FF93C091E900CF708091EC00E2
:1052D000D82FD17080FDD0E81092E9008091F000C5
:1052E000877F8093F00078940E947B261092E900DB
:1052F0008091F00088608093F000CD2BCF70C09338
:10530000E900FF91EF91DF91CF91BF91AF919F9114
:105310008F917F916F915F914F913F912F910F905E
:105320000FBE0F901F901895E8EDF0E080818E7F02
:1053300080831092E2001092DA001092E100A0EE59
:10534000B0E08C9181608C9380818F77808319BCD1
:10535000A7EDB0E08C918E7F8C9380818F7E8083CF
:105360001092000608952091E4003091E50095E642
:105370004091EC00842F817040FF22C08091E800B2
:1053800080FD1CC08091C805882391F0853091F084
:105390008091EB0085FD10C04091E4005091E50044
:1053A0004217530729F39A01915011F784E00895A9
:1053B00082E0089583E0089581E0089580E00895F3
:1053C0004091E80042FFDECF08958091CA0587FF33
:1053D00011C08091E80082FD05C08091C80581114F
:1053E000F8CF11C08091E8008B770BC08091C80581
:1053F000882349F08091E80080FFF8CF8091E80091
:105400008E778093E8000895982F973058F5909301
:10541000E900981739F07091EC002091ED0050915F
:10542000F00003C0242F762F50E021FF19C03091E7
:10543000EB003E7F3093EB003091ED003D7F3093E9
:10544000ED003091EB0031603093EB007093EC0095
:105450002093ED005093F0002091EE0027FF07C04D
:105460009F5FD3CF8F708093E90081E0089580E043
:105470000895CF92DF92EF92FF920F931F93CF93F5
:10548000DF93C8EDD0E088818F7E8883E7EDF0E080
:1054900080818160808384E082BF81E08093000608
:1054A00088818E7F888302EE10E0F80110821092CE
:1054B000DA0081EEC82ED12CF601108288818F7718
:1054C000888388818068888388818F7D888319BCE0
:1054D0001092C8051092C9051092C7051092C60512
:1054E00090EEE92EF12CF70180818B7F80838881FB
:1054F0008160888342E060E080E00E94042AF60137
:1055000080818E7F8083F8018081816080838081AB
:1055100088608083F70180818E7F808388818061AD
:105520008883DF91CF911F910F91FF90EF90DF90D3
:10553000CF9008951F920F920FB60F9211242F93C0
:105540003F934F935F936F937F938F939F93AF930B
:10555000BF93EF93FF938091E10082FF09C0809198
:10556000E20082FF05C08091E1008B7F8093E10023
:105570008091DA0080FF2AC08091D80080FF26C089
:105580008091DA008E7F8093DA008091D90080FFCD
:1055900018C080E189BD82E189BD09B400FEFDCF5C
:1055A00081E08093C8058091000681110FC00E94A0
:1055B00094290E94392A8091E20084608093E2005D
:1055C00005C019BC1092C805109200068091E10038
:1055D00080FF17C08091E20080FF13C08091E2003D
:1055E0008E7F8093E2008091E20080618093E200F0
:1055F0008091D80080628093D80019BC85E08093A8
:10560000C8058091E10084FF34C08091E20084FFEE
:1056100030C080E189BD82E189BD09B400FEFDCFC3
:105620008091D8008F7D8093D8008091E1008F7E9B
:105630008093E1008091E2008F7E8093E200809170
:10564000E20081608093E2008091C905882311F017
:1056500084E007C08091E30087FD02C081E001C0C3
:1056600083E08093C8051092BB050E940D2C0E9418
:10567000770F8091E10083FF27C08091E20083FFD4
:1056800023C08091E100877F8093E10082E08093D6
:10569000C8051092C9058091E1008E7F8093E100DA
:1056A0008091E2008E7F8093E2008091E200806131
:1056B0008093E20042E060E080E00E94042A809152
:1056C000F00088608093F000FF91EF91BF91AF915F
:1056D0009F918F917F916F915F914F913F912F910A
:1056E0000F900FBE0F901F9018952091D00530910C
:1056F000D1052617370748F06115710539F4209157
:10570000E8002E772093E80001C0B90140E0611560
:105710007105A9F12091C805222309F443C0253061
:1057200009F442C02091E80023FD40C02091E80028
:1057300022FD32C02091E80020FFE9CF4091F30024
:105740002091F20030E0342BFC01CF01611571058E
:1057500059F02830310540F481918093F100615077
:1057600071092F5F3F4FF1CF41E02830310509F03B
:1057700040E02091E8002E772093E800C8CF411147
:10578000C9CF0AC08091C805882361F0853061F0D7
:105790008091E80083FD0AC08091E80082FFF2CF8B
:1057A00080E0089582E0089583E0089581E00895FF
:1057B0000E948822292F2F7092959F70E92FF0E088
:1057C0003297EE30F105B8F4ED56FF4F0C9471327C
:1057D000803F99F018F4803E70F40FC0843F59F474
:1057E0000CC0803E50F0813F31F407C0822F869577
:1057F00086958695089580E0089581E00895109239
:10580000B6051092B5050E94192280E090E00E9432
:10581000610F80E090E00C944B0F86E0E2E5F5E04C
:10582000DF011D928A95E9F70C94FF2B882341F044
:1058300080959091BB0589238093BB050C94192218
:105840000895882339F09091BB05892B8093BB057F
:105850000C94192208958823A9F19CEF980F913A8E
:1058600060F4E2E5F5E096E09E0F2081281301C088
:10587000108231969E13F9CF14C090E2980F9830A1
:1058800090F4877021E030E0A90102C0440F551F59
:105890008A95E2F7CA0180959091BB058923809390
:1058A000BB050C9419229BE5980F933020F480E0FF
:1058B00090E00C94610F885A873120F480E090E0EA
:1058C0000C944B0F0895882309F4C4C09CEF980FE3
:1058D000913A30F4682F80E595E00E94AE2113C024
:1058E00090E2980F983088F4877021E030E0A901A9
:1058F00002C0440F551F8A95E2F7CA019091BB057B
:10590000892B8093BB050C9419229BE5980F93304B
:1059100070F4853A29F0863A31F083E890E005C0CA
:1059200081E890E002C082E890E00C94610F98E575
:10593000980F973108F08EC0883A09F445C0893A2B
:1059400009F445C08A3A09F445C08B3A09F445C0C8
:105950008C3A09F445C08B3B09F445C08C3B09F4F3
:1059600045C08D3A09F445C0803B09F445C08E3AE4
:1059700009F445C08F3A09F445C0813B09F445C09C
:10598000823B09F445C0833B09F445C0843B09F4DC
:1059900045C0853B09F445C0863B09F445C0873BBB
:1059A00009F445C0883B09F445C0893B09F445C06A
:1059B0008D3B09F445C08E3B09F445C08A3B09F490
:1059C00045C080E090E044C082EE90E041C089EEA6
:1059D00090E03EC08AEE90E03BC085EB90E038C09E
:1059E00086EB90E035C083EB90E032C084EB90E032
:1059F0002FC087EB90E02CC08CEC90E029C08DECA0
:105A000090E026C083E891E023C08AE891E020C0BE
:105A100082E991E01DC084E991E01AC081E292E040
:105A200017C083E292E014C084E292E011C085E2E4
:105A300092E00EC086E292E00BC087E292E008C0DE
:105A40008FE690E005C080E790E002C08AE292E035
:105A50000C944B0F08958F929F92AF92BF92CF926A
:105A6000DF92EF92FF92CF93DF93EC01688179810F
:105A70008A819B81611571058105910521F464E29C
:105A800079ED8BE597E02DE133EF41E050E00E94A6
:105A9000CF2D49015A019B01AC01A7EAB1E40E9454
:105AA000EE2D6B017C01ACEEB4EFA50194010E94D8
:105AB000FC2DDC01CB018C0D9D1DAE1DBF1DB7FF64
:105AC00003C00197A109B04888839983AA83BB8347
:105AD0009F77DF91CF91FF90EF90DF90CF90BF90B5
:105AE000AF909F908F9008950E942B2D089580E095
:105AF00091E00E942B2D0895A0E0B0E0809300017A
:105B000090930101A0930201B09303010895F999C4
:105B1000FECF92BD81BDF89A992780B50895A6E180
:105B2000B0E044E050E00C94C12DA8E1B0E042E0C8
:105B300050E00C94C12D262FF999FECF92BD81BD66
:105B4000F89A019700B4021639F01FBA20BD0FB6BB
:105B5000F894FA9AF99A0FBE08950396272F0E9497
:105B60009C2D0E949B2D252F0E949C2D242F0C9450
:105B70009C2D0196272F0E949C2D0C949B2DDC01BF
:105B8000CB01FC01F999FECF06C0F2BDE1BDF89A48
:105B9000319600B40D9241505040B8F70895052E4B
:105BA00097FB1EF400940E94E62D57FD07D00E943B
:105BB000012E07FC03D04EF40C94E62D5095409531
:105BC000309521953F4F4F4F5F4F089590958095A9
:105BD000709561957F4F8F4F9F4F08950E94232EA0
:105BE000A59F900DB49F900DA49F800D911D112431
:105BF0000895B7FF0C94EE2D0E94EE2D821B930B9F
:105C00000895A1E21A2EAA1BBB1BFD010DC0AA1FFD
:105C1000BB1FEE1FFF1FA217B307E407F50720F015
:105C2000A21BB30BE40BF50B661F771F881F991F90
:105C30001A9469F760957095809590959B01AC01D9
:105C4000BD01CF010895A29FB001B39FC001A39FE2
:105C5000700D811D1124911DB29F700D811D1124A5
:105C6000911D08955058BB27AA270E944A2E0C94D4
:105C70001E300E94103038F00E94173020F039F4A6
:105C80009F3F19F426F40C94E62F0EF4E095E7FB01
:105C90000C94E02FE92F0E942F3058F3BA176207B7
:105CA00073078407950720F079F4A6F50C9451301A
:105CB0000EF4E0950B2EBA2FA02D0B01B901900127
:105CC0000C01CA01A0011124FF27591B99F0593F6B
:105CD00050F4503E68F11A16F040A22F232F342FB3
:105CE0004427585FF3CF469537952795A795F04001
:105CF0005395C9F77EF41F16BA0B620B730B840B16
:105D0000BAF09150A1F0FF0FBB1F661F771F881FCD
:105D1000C2F70EC0BA0F621F731F841F48F4879525
:105D200077956795B795F7959E3F08F0B0CF939517
:105D3000880F08F09927EE0F9795879508950E9490
:105D4000BC2F08F481E008950E94B82E0C941E30F8
:105D50000E94173058F00E94103040F029F45F3F45
:105D600029F00C94E02F51110C9452300C94E62F32
:105D70000E942F3068F39923B1F3552391F3951BBB
:105D8000550BBB27AA2762177307840738F09F5F5C
:105D90005F4F220F331F441FAA1FA9F335D00E2EC9
:105DA0003AF0E0E832D091505040E695001CCAF736
:105DB0002BD0FE2F29D0660F771F881FBB1F2617F9
:105DC00037074807AB07B0E809F0BB0B802DBF01D0
:105DD000FF2793585F4F3AF09E3F510578F00C949F
:105DE000E02F0C9452305F3FE4F3983ED4F3869555
:105DF00077956795B795F7959F5FC9F7880F911DC0
:105E00009695879597F90895E1E0660F771F881FAB
:105E1000BB1F621773078407BA0720F0621B730B5E
:105E2000840BBA0BEE1F88F7E095089529F416F05D
:105E30000C94E02F0C9451300C94E62F0E943730D4
:105E4000A8F39638A0F707F80F92E8942BE33AEA04
:105E500048EB5FE70E94E9300F920F920F924DB727
:105E60005EB70F920E949F30E2E4F1E00E94E92FBA
:105E70004F915F91EF91FF91E595EE1FFF1F49F064
:105E8000FE57E0684427EE0F441FFA95E1F741956D
:105E9000550B0E9469300F9007FE0C945D300895F9
:105EA0000E94373088F09F5798F0B92F9927B75143
:105EB000B0F0E1F0660F771F881F991F1AF0BA95AE
:105EC000C9F714C0B13091F00E945130B1E008958B
:105ED0000C945130672F782F8827B85F39F0B93F7D
:105EE000CCF3869577956795B395D9F73EF4909561
:105EF0008095709561957F4F8F4F9F4F0895E894DF
:105F000009C097FB3EF490958095709561957F4F01
:105F10008F4F9F4F9923A9F0F92F96E9BB279395AF
:105F2000F695879577956795B795F111F8CFFAF4BF
:105F3000BB0F11F460FF1BC06F5F7F4F8F4F9F4FF0
:105F400016C0882311F096E911C0772321F09EE84E
:105F5000872F762F05C0662371F096E8862F70E0B4
:105F600060E02AF09A95660F771F881FDAF7880F8E
:105F70009695879597F90895990F0008550FAA0BE4
:105F8000E0E8FEEF16161706E807F907C0F012164C
:105F90001306E407F50798F0621B730B840B950B4F
:105FA00039F40A2661F0232B242B252B21F40895A4
:105FB0000A2609F4A140A6958FEF811D811D089541
:105FC00097F99F6780E870E060E008959FEF80ECAC
:105FD0000895DF93CF931F930F93FF92EF92DF9279
:105FE0007B018C01689406C0DA2EEF010E94E63036
:105FF000FE01E894A5912591359145915591A6F31F
:10600000EF010E944A2EFE019701A801DA9469F778
:10601000DF90EF90FF900F911F91CF91DF91089546
:1060200000240A9416161706180609060895002477
:106030000A9412161306140605060895092E0394F1
:10604000000C11F4882352F0BB0F40F4BF2B11F465
:1060500060FF04C06F5F7F4F8F4F9F4F089557FDC4
:106060009058440F551F59F05F3F71F04795880FC6
:1060700097FB991F61F09F3F79F08795089512165D
:1060800013061406551FF2CF4695F1DF08C0161609
:1060900017061806991FF1CF8695710561050894BA
:1060A0000895E894BB2766277727CB0197F90895D1
:1060B0000E94BC2F08F48FEF08959B01AC0160E0B3
:1060C00070E080E89FE30C94A42E0C94E02F0C94D5
:1060D00098310E943730D8F39923C9F3940F511D9A
:1060E000A3F39150504094F059F0882332F0660F9A
:1060F000771F881F91505040C1F79E3F51052CF7E4
:10610000880F911D9695879597F908955F3FACF09C
:10611000983E9CF0BB27869577956795B79508F4D0
:10612000B1609395C1F7BB0F58F711F460FFE8CF4A
:106130006F5F7F4F8F4F9F4FE3CF0C945230FA0128
:10614000DC01AA0FBB1F9B01AC01BF5728F422271B
:1061500033274427507820C0B75190F4AB2F002448
:10616000469537952795011CA395D2F3002071F031
:10617000220F331F441FB395DAF30ED00C94322E46
:1061800061307105A0E88A07B94630F49B01AC0183
:106190006627772788279078309621F020833183EF
:1061A0004283538308950E94E6300C941E300E946F
:1061B000103038F00E94173020F0952311F00C9425
:1061C000E02F0C94E62F11240C9452300E942F30B3
:1061D00070F3959FC1F3950F50E0551F629FF0013A
:1061E000729FBB27F00DB11D639FAA27F00DB11D53
:1061F000AA1F649F6627B00DA11D661F829F2227DC
:10620000B00DA11D621F739FB00DA11D621F839F62
:10621000A00D611D221F749F3327A00D611D231F38
:10622000849F600D211D822F762F6A2F11249F5786
:1062300050409AF0F1F088234AF0EE0FFF1FBB1F89
:10624000661F771F881F91505040A9F79E3F510548
:1062500080F00C94E02F0C9452305F3FE4F3983EB2
:10626000D4F3869577956795B795F795E7959F5FF2
:10627000C1F7FE2B880F911D9695879597F9089584
:10628000FA01EE0FFF1F309621053105A1F16115CE
:10629000710561F48038BFE39B0749F16894903839
:1062A000810561F08038BFEF9B0741F099234AF5E3
:1062B000FF3FE1053105210519F1E8940894E795C0
:1062C000D901AA2329F4AB2FBE2FF85FD0F310C059
:1062D000FF5F70F4A695E0F7F73950F019F0FF3A38
:1062E00038F49F779F930DD00F9007FC9058089536
:1062F00046F00C94E62F60E070E080E89FE308959C
:106300004FE79F775F934F933F932F930E94ED3119
:106310002F913F914F915F910E94D3300C941E2F8B
:106320009F930E94A8310F9007FCEE5F0C94D1312F
:106330009F3F31F0915020F4879577956795B795F9
:10634000880F911D9695879597F908950C94E62FDF
:106350000E943730D8F3E894E0E0BB279F57F0F075
:106360002AED3FE049EC06C0EE0FBB0F661F771F1A
:10637000881F28F0B23A62077307840728F0B25AE0
:10638000620B730B840BE3959A9572F7803830F4A7
:106390009A95BB0F661F771F881FD2F790480C9401
:1063A0009A31EF93E0FF07C0A2EA2AED3FE049EC03
:1063B0005FEB0E944A2E0E941E300F90039401FC56
:1063C0009058EAE6F1E00C94353216F00C949831CE
:1063D0000C94E62F68940C94E02F0E943730A8F3B9
:1063E0009923C1F3AEF3DF93CF931F930F93FF92E3
:1063F000C92FDD2788232AF02197660F771F881F72
:10640000DAF720E030E040E85FEB9FE3883920F0E6
:10641000803E38F021968F770E94332EE8E8F1E035
:1064200004C00E94332EE5EBF1E00E94E92F8B01BE
:10643000BE01EC01FB2E6F5771097595771F880B14
:10644000990B0E94812F28E132E741E35FE30E942C
:10645000E630AF2D9801AE01FF900F911F91CF91C3
:10646000DF910E944A2E0C941E309F938F937F934E
:106470006F93FF93EF939B01AC010E94D330EF9198
:10648000FF910E94E92F2F913F914F915F910C94C2
:10649000D330AA1BBB1B51E107C0AA1FBB1FA61705
:1064A000B70710F0A61BB70B881F991F5A95A9F7BD
:1064B00080959095BC01CD01089597FB072E16F4A9
:1064C000009407D077FD09D00E94493207FC05D01F
:1064D0003EF4909581959F4F0895709561957F4FFB
:1064E0000895EE0FFF1F0590F491E02D0994FC0133
:1064F0004150504030F001900616D1F73197CF014E
:0C6500000895882799270895F894FFCF8C
:10650C00010000000000DC43000040400000DC43C0
:10651C000000803F0000DC430AA7CF44000000418C
:10652C000000DC440000004100000000000080403E
:10653C0052D02445000000410000000000008040C3
:10654C005CFF384500000041000000000000804066
:10655C0052D02445000000410AA7CF44000000415E
:10656C000000DC44000000410000000000008040FE
:10657C0052D0244500004041000000000000804043
:10658C000AA74F45000040410AA7CF440000004134
:10659C000000DC44000000410000000000008040CE
:1065AC0052D024450000804100005C440000804132
:1065BC005C978A440000804152D0A4440000804182
:1065CC000000DC44000080410000DC44000000417D
:1065DC000AA7CF44000000415CFFB8440000004112
:1065EC0052D0A444000000411FD592440000004149
:1065FC005C978A440000004148F176440000004159
:10660C0000005C440000004100005C44000080413C
:10661C001F1569440000804148F176440000804118
:10662C0000D08244000080415C978A440000804185
:10663C00A4D024440000804100005C440000804150
:10664C001FD59244000080415CFFC3440000804190
:10665C0000000000000000005CFF4344000080418B
:10666C001FD59244000080410000DC4400008041B2
:10667C0052D02445000080410000000000000000C2
:10668C0000005C440000804148F1764400008041E9
:10669C005C978A44000080411FD5924400008041E1
:1066AC0052D0A4440000804103640052D024450021
:1066BC000000410000DC440000004152D0A4440022
:1066CC0000404100005C440000004100005C4400BC
:1066DC0000004148F176440000C04000005C4400DA
:1066EC0000C04048F176440000C04000005C44000B
:1066FC0000C0400552D0A444000000410000DC441E
:10670C000000004152D02445000040410000003FF1
:10671C000100005C44000000410000DC440000006B
:10672C00410000DC440000004100005C440000001B
:10673C004100005C440000004148F1764400000038
:10674C00415C978A44000000411FD5924400000030
:10675C004152D0A444000000415CFFB8440000004A
:10676C00410AA7CF44000000410000DC44000000B7
:10677C004100005C440000004148F17644000000F8
:10678C00415C978A44000000411FD59244000000F0
:10679C004152D0A444000000415CFFB8440000000A
:1067AC00410AA7CF44000000410000DC4400000077
:1067BC00410000DC44000000410AA7CF4400000067
:1067CC00415CFFB8440000004152D0A444000000DA
:1067DC00411FD59244000000415C978A44000000A0
:1067EC004148F176440000004100005C4400000088
:1067FC004100005C440000004148F1764400000078
:10680C00415C978A44000000411FD592440000006F
:10681C004152D0A444000000415CFFB84400000089
:10682C00410AA7CF44000000410000DC44000000F6
:10683C004101191A1B1C1D1E1F202122010A0504CF
:10684C0006050402050102691CE01C681CAA1C6CEC
:10685C001C010002040507090B0C0E10111315176F
:10686C00181A1C1D1F2123242628292B2D2F3032CA
:10687C00343537393B946697C600000000F4F5F6C2
:04688C00F73133327B
:00000001FF
